:040000006EEF2EF081
:1000080000C023F001C022F002C021F003C020F09C
:1000180004C01FF005C01EF006C01DF007C01CF08C
:1000280008C01BF009C01AF00AC019F00BC018F07C
:100038000CC017F00DC016F00EC015F0E1CF24F07B
:10004800E2CF25F0F2A851D0F2A24FD0010E010163
:100058005D27000E5E235F2360235DC100F05EC153
:1000680001F05FC102F060C103F012EC0FF09A0ECC
:10007800046ED90E056E580E066E870E076E5EEC7E
:100088000AF000C0A4F101C0A5F102C0A6F103C0A6
:10009800A7F1030E046E000E056E066E076E5DC1B5
:1000A80000F05EC101F05FC102F060C103F01CEC1A
:1000B8000BF008C000F009C001F00AC002F00BC044
:1000C80003F0000E046E031808E10450021805E15D
:1000D8000450011802E10050000AD8B4897881B6AA
:1000E80003D00101A26BA36BF2929DA024D09EA025
:1000F80022D0DB0ECE6E0B0ECF6E010E0201332521
:10010800006E000E3421016E00C033F201C034F2DB
:1001180001014C510201345D04E101014B5102011E
:10012800335D08E3336B346B010E0101C46F000EBD
:10013800C56F9D909E909DAA5ED09EAA5CD05AECF9
:1001480026F000C09BF2ABA215D0AB98AB885AEC56
:1001580026F000C09BF25AEC26F000C09BF2010E7C
:1001680001019025006E000E9121016E00C090F1F2
:1001780001C091F1ABA40DD00101AB9EAB8E010E75
:100188009025006E000E9121016E00C090F101C013
:1001980091F102019B510D0A15E1010E316F000E1C
:1001A800326FD40E0101CA25E16E010ECB21E26E39
:1001B800E66ACAC1D0F1CBC1D1F1CA6BCB6B0201DF
:1001C8009B6B19D0316B326BD40E0101CA25E16EDD
:1001D800010ECB21E26E9BC2E6FFCAC1D0F1CBC1B2
:1001E800D1F1010ECA25006E000ECB21016E00C0B0
:1001F800CAF101C0CBF123C000F022C001F021C038
:1002080002F020C003F01FC004F01EC005F01DC09E
:1002180006F01CC007F01BC008F01AC009F019C08E
:100228000AF018C00BF017C00CF016C00DF015C07E
:0C0238000EF024C0E1FF25C0E2FF110021
:10024400C7B409D01F0EC514016E0150000A03E1A2
:0A025400010E006E01D0006A1200D6
:0E025E00026A016A006A086A036A000E120052
:10026C000B840BAE41EF01F0010E036E026A016AC2
:0A027C00006A0A360232FF0E12007B
:100286000B820BAE4DEF01F003680268016800684F
:080296000A360232FF0E1200CD
:08029E000AAE029E000E1200E0
:1002A6009E9699C2C9FFC7A401D0FDD79EB601D0BC
:1002B600FDD7C5BC02D0006A03D0C584020E006E0D
:0202C600120024
:0402C800C5841200D7
:1002CC000CB0A8EF01F00CA24EEF02F00E6A000E7B
:1002DC000264BFEF01F0F00E0214D8A48AEF01F013
:1002EC00023A01380F0B02260138F00B016E003870
:1002FC000F0B01260038F00B006E08380F0B002690
:10030C000838F00B086E0E84D89002BEA3EF01F0F3
:10031C0008360036013602360E2A02BEA3EF01F073
:10032C0008360036013602360E2A02BEA3EF01F063
:10033C0008360036013602360E2A0E50036444EF9E
:10034C0002F0035E0BBC08AE49EF02F0D880800EC1
:10035C0008640030000E002201220222D8A049EFCE
:10036C0002F0023201320032034A4EEF02F049EF42
:10037C0002F001C002F000C001F008C000F0086AF1
:10038C00000E0E860264F6EF01F0F00E0214D8A4F3
:10039C00DEEF01F0023A01380F0B02260138F00BA8
:1003AC00016E00380F0B01260038F00B006E0E8426
:1003BC00D89002BEA3EF01F00036013602360E2AA9
:1003CC0002BEA3EF01F00036013602360E2A02BE41
:1003DC00A3EF01F00036013602360E2AA3EF01F02E
:1003EC0001C002F000C001F0006A000E0E960E88EB
:1003FC00026423EF02F0F00E0214D8A40EEF02F008
:10040C00023A01380F0B02260138F00B016E0E84F4
:10041C00D89002BEA3EF01F0013602360E2A02BEBE
:10042C00A3EF01F0013602360E2A02BEA3EF01F053
:10043C00013602360E2AA3EF01F001C002F0016A68
:10044C00000E0E86026453EF02F0F00E0214D8A4D4
:10045C0032EF02F0023A0E84D89002BEA3EF01F004
:10046C0002360E2A02BEA3EF01F002360E2A02BE9D
:10047C00A3EF01F002360E2AA3EF01F0010E0C6E71
:10048C00EFDE56EF02F0020E0C6E03DF56EF02F0B9
:10049C00040E0C6EF2DE56EF02F0080E0C6ED9DE76
:0204AC0012003C
:1004AE000201996B9A6B9A51120802E199518E08CA
:1004BE0008E3C1DE005201E004D00201994B9A2BF1
:1004CE00F2D70201120E9A5D02E18F0E995D03E3DF
:1004DE007B0E006E05D0C580C5A001D0FDD7006A89
:0204EE001200FA
:1004F000DEDF96C299F2D7DE00C098F297C299F279
:0E050000D2DE00C098F2E0DE98C200F01200D9
:10050E00086A080E0C6E003408360450085ED8B027
:0E051E0002D00826D89000360C2EF5D7120019
:10052C000134083609360450085E0550D8A0053C45
:10053C00095E003601360F0E0C6E01340836093692
:10054C00045000A006D0085E0550D8A0053C095EFA
:10055C0005D008260550D8B0053C092600360136D2
:10056C000C2EEBD700B006D0045008260550D8B09E
:08057C00053C092600001200F5
:10058400025006180E6E086A096A0B6A0350076463
:10059400B5EF03F006500A6E068E028E03500B6E02
:1005A4000750036E000E0B6405EF03F00B50075E5B
:1005B400D8B4A6EF03F0070E076474EF03F0075EE8
:1005C40000C008F001C000F002C001F0026A074E4A
:1005D400A6EF03F0076449EF03F0075E00C008F0DC
:1005E40001C000F0016A074EA6EF03F0076427EF8D
:1005F40003F0075E00C008F0006A074EA6EF03F0A0
:1006040007640EEF03F00AC002F005C001F004C055
:1006140000F0086ACFEF04F0030E076419EF03F04B
:10062400075E08380F0B086E074EA6EF03F0D8904C
:100634000832074EA6EF03F0D8900832074EA6EF13
:1006440003F0D8900832A6EF03F0030E076438EFE6
:1006540003F0075E08380F0B086E0038F00B08260D
:1006640000380F0B006E074EA6EF03F0D89000324F
:100674000832074EA6EF03F0D89000320832074E36
:10068400A6EF03F0D89000320832A6EF03F0030E71
:10069400076460EF03F0075E08380F0B086E00383C
:1006A400F00B082600380F0B006E0138F00B002603
:1006B40001380F0B016E074EA6EF03F0D8900132FC
:1006C40000320832074EA6EF03F0D8900132003210
:1006D4000832074EA6EF03F0D890013200320832F8
:1006E400A6EF03F0030E076491EF03F0075E0838EA
:1006F4000F0B086E0038F00B082600380F0B006E45
:100704000138F00B002601380F0B016E0238F00B94
:10071400012602380F0B026E074EA6EF03F0D890A5
:100724000232013200320832074EA6EF03F0D890AD
:100734000232013200320832074EA6EF03F0D8909D
:100744000232013200320832096A000E0EAE9AEF0C
:1007540004F0081E001E011E021E082A00220122A7
:1007640002229AEF04F00750D8A4BBEF03F0CFEFB6
:1007740004F0096A02C00AF0028E068E0750035C78
:10078400076ED8B48DEF04F0070E07645BEF04F036
:10079400075E0450096E0550046E0650056E066A25
:1007A400074E8DEF04F0070E076430EF04F0075E88
:1007B4000450096E0550046E056A074E8DEF04F06F
:1007C400070E07640EEF04F0075E0450096E046A16
:1007D400074E8DEF04F0070E0764F5EF03F00AC02F
:1007E40002F0CFEF04F0030E076400EF04F0075E9D
:1007F40009380F0B096E074E8DEF04F0D8900932BB
:10080400074E8DEF04F0D8900932074E8DEF04F0B7
:10081400D89009328DEF04F0030E07641FEF04F043
:10082400075E09380F0B096E0438F00B09260438EB
:100834000F0B046E074E8DEF04F0D890043209328A
:10084400074E8DEF04F0D89004320932074E8DEF35
:1008540004F0D890043209328DEF04F0030E0764DB
:1008640047EF04F0075E09380F0B096E0438F00BEC
:10087400092604380F0B046E0538F00B04260538DE
:100884000F0B056E074E8DEF04F0D890053204323D
:100894000932074E8DEF04F0D89005320432093244
:1008A400074E8DEF04F0D8900532043209328DEFF3
:1008B40004F0030E076478EF04F0075E09380F0BA9
:1008C400096E0438F00B092604380F0B046E053842
:1008D400F00B042605380F0B056E0638F00B0526C1
:1008E40006380F0B066E074E8DEF04F0D8900632D3
:1008F400053204320932074E8DEF04F0D8900632E7
:10090400053204320932074E8DEF04F0D8900632D6
:10091400053204320932086A000E0EAE9AEF04F072
:10092400091E041E051E061E092A0422052206228B
:1009340009500826045000220550012206500222C4
:100944000EBEB1EF04F0D8A0C0EF04F002320132C1
:1009540000320832033EC0EF04F0CAEF04F0D8B00E
:10096400C5EF04F0000E081E001E011E021E082A18
:100974000022012202220A7EC5EF04F0010E0C6E51
:10098400A3DCD1EF04F0020E0C6E9EDCD1EF04F078
:10099400040E0C6E76DCD1EF04F0000E0C6E120027
:1009A400086A096A000E0762036457EF05F00250F3
:1009B40006180A6E075003267E0ED8A0E8EF04F04E
:1009C400035ED8B05CEF05F0ECEF04F0035ED8A052
:1009D40061EF05F0028E068E02C00EF001C00BF02E
:1009E40000C00DF000500402F4CF0CF001500502D9
:1009F400F4CF00F0F3CF08F00402F3500C26F450C7
:100A04000822000E00220D500502F3500C26F4506B
:100A14000822000E002202500402F3500826F4506B
:100A2400002202500502016A000E0122F350002642
:100A3400F45001220D500602F3500826F45000220F
:100A4400026A000E012202220B500602F350002615
:100A5400F4500122000E02220E500602F350012629
:100A6400F450022202BE3FEF05F00836003601368C
:100A740002360306D8B461EF05F052EF05F0D880D2
:100A8400800E08640030000E002201220222D8A049
:100A940052EF05F0023201320032034A5CEF05F0F6
:100AA4000AAE029E000E64EF05F0010E2FEC01F079
:100AB40064EF05F0020E43EC01F064EF05F0040E60
:060AC40036EC01F0120007
:080ACA000B6A0B86FF0E1200FF
:100AD2000B800BAE75EF05F0026A0AAEFF0E026ED6
:0C0AE200016E006E0A360232FF0E120098
:100AEE000D6A086A0050D8B4000C04180A6E0ABECB
:100AFE000D1E0B6A04AE02D0041E042A00AE02D0F4
:100B0E00001E002A005004100A6E0ABE1FD00450A8
:100B1E00085E003600340836045008260036060EED
:100B2E000C6E00340836045000B0085E00A0082693
:100B3E0000360C2EF6D700A008260BB015D00DAE41
:100B4E00000C001E002A081E082A000C04AE09D054
:100B5E0000BE04D00050086E006AF1D7006A002A69
:100B6E00000C001E0B2AD3D7082A0450085CD8A408
:0E0B7E00E6D7086A002A00AEE2D7FF0C12008C
:100B8C0002019151390806E3300E915D03E3010E29
:080B9C00006E01D0006A120096
:100BA40003500718D8A4E6EF05F002500618D8A49D
:100BB400E6EF05F001500518D8A4E6EF05F0005063
:0E0BC4000418D8B4D8841200D894120012007D
:100BD2009E96C5869EB601D0FDD7C9CF01F002010F
:100BE2009151000A02E1C58A01D0C59A9E96C58834
:0C0BF2009EB601D0FDD701C000F012003B
:100BFE000B6A0C6A086A0350D8B483EF06F002C081
:100C0E000AF0028E9E0E035E03AE73EF06F0036CC7
:100C1E00080E035CD8A040EF06F0036E083600C045
:100C2E0008F001C000F002C001F0026A080E035C79
:100C3E00D8A040EF06F0036E083600C008F001C0E1
:100C4E0000F0016A080E035CD8A040EF06F0036EB8
:100C5E00083600C008F0006A080E035CD8A040EF0A
:100C6E0006F0036E0836086A0350D8A4D8904CEFED
:100C7E0006F00350D8B44CEF06F0D8900232013291
:100C8E0000320832032E44EF06F00BBC08A05DEFD5
:100C9E0006F0D8A05DEF06F0082AD8B4002AD8B422
:100CAE00012AD8B4022A02BE87EF06F00AAE83EFFD
:100CBE0006F0021E011E001E081E082AD8B4002AC5
:100CCE00D8B4012AD8B4022A83EF06F0026A016A68
:100CDE00006A086A83EF06F00B800BAE8DEF06F00C
:100CEE00026A0AAE8DEF06F0026E016E006E086E9D
:100CFE000A3602328DEF06F00C6A000E8EEF06F009
:100D0E00010E0C6E000EDEDE8EEF06F0FF0E0250B0
:100D1E00036E0150026E0050016E0850006E1200FC
:100D2E000450000A08E10550000A05E1FF0E006EAE
:100D3E007F0E016E58D00D6A096A086A01500010C4
:100D4E00D8B4000C015005180A6E0ABE0D1E0B6AAF
:100D5E0005AE05D0041E051E042AD8B4052A01AE20
:100D6E0005D0001E011E002AD8B4012A015005101C
:100D7E000A6E0ABE10D096EC02F00BB020D00DAE6B
:100D8E00000C001E011E002AD8B4012A081E091EDE
:100D9E00082AD8B4092A000C05AE0DD001BE07D022
:100DAE000150096E0050086E016A006AE8D7016AA8
:100DBE00006A002A000C011E001E0B2ADDD7082A2D
:100DCE00D8B4092A0450085CD8A4D9D70550095CB8
:100DDE00D8A4D5D7096A086A002AD8B4012A01AE68
:080DEE00CED70000FF0C12003B
:100DF600800E02019119006E800E000A005CD8B0C8
:100E060064D191510008016E01C091F2800E011863
:100E1600006E800E6E0A005CD8A0BAD0640E046E16
:100E260091C200F061DE120E0024056E000E00BEB7
:100E3600FF0E066E000E062205C000F006C001F089
:100E4600000E06BEFF0E026E036E003600900136DF
:100E56000236033600360090013602360336350E6A
:100E66000024F66E6D0E0120F76E000E0220F86E5D
:100E76000900F5CF92F20900F5CF93F20900F5CFFC
:100E860094F20900F5CF95F2640E046E91C200F05B
:100E96002BDE08C000F00A0E046E26DE090E0024C2
:100EA600056E000E00BEFF0E066E000E062205C081
:100EB60000F006C001F0000E06BEFF0E026E036EC5
:100EC60000360090013602360336003600900136B1
:100ED60002360336350E0024F66E6D0E0120F76ECF
:100EE600000E0220F86E0900F5CF00F00900F5CFDC
:100EF60001F00900F5CF02F00900F5CF03F092C228
:100F060004F093C205F094C206F095C207F047DDDF
:100F160000C092F201C093F202C094F203C095F2AF
:100F26000A0E046E91C200F0DFDD08C000F000C0BA
:100F360001F0000E00BEFF0E026E036E046E013657
:100F46000190023603360436013601900236033626
:100F56000436350E0124F66E6D0E0220F76E000E75
:100F66000320F86E0900F5CF00F00900F5CF01F077
:100F76000900F5CF02F00900F5CF03F092C204F0A4
:100F860093C205F094C206F095C207F008DDFED1C3
:100F9600800E0A0A006E800E9119005C6EE20A0E3F
:100FA600046E91C200F0A0DD090E0024056E000E4D
:100FB60000BEFF0E066E000E062205C000F006C03B
:100FC60001F0000E06BEFF0E026E036E00360090A4
:100FD60001360236033600360090013602360336F5
:100FE600350E0024F66E6D0E0120F76E000E0220FF
:100FF600F86E0900F5CF92F20900F5CF93F20900D9
:10100600F5CF94F20900F5CF95F20A0E046E91C25F
:1010160000F06ADD08C000F000C001F0000E00BE5E
:10102600FF0E026E036E046E013601900236033621
:10103600043601360190023603360436350E012495
:10104600F66E6D0E0220F76E000E0320F86E090094
:10105600F5CF00F00900F5CF01F00900F5CF02F059
:101066000900F5CF03F092C204F093C205F094C2D2
:1010760006F095C207F093DC89D191C200F0000E0C
:1010860091BFFF0E016E026E036E003600900136B0
:101096000236033600360090013602360336350E28
:1010A6000024F66E6D0E0120F76E000E0220F86E1B
:1010B6000900F5CF00F00900F5CF01F00900F5CFE2
:1010C60002F00900F5CF03F061D1800E9119006E90
:1010D600800E6E0A005CD8A0BCD0640E046E91C26D
:1010E60000F002DD120E0024056E000E00BEFF0E9B
:1010F600066E000E062205C000F006C001F0000EC6
:1011060006BEFF0E026E036E0036009001360236F2
:10111600033600360090013602360336690E002487
:10112600F66E6D0E0120F76E000E0220F86E0900B5
:10113600F5CF92F20900F5CF93F20900F5CF94F2BC
:101146000900F5CF95F2640E046E91C200F0CCDC76
:1011560008C000F00A0E046EC7DC090E0024056EF6
:10116600000E00BEFF0E066E000E062205C000F041
:1011760006C001F0000E06BEFF0E026E036E0036BC
:1011860000900136023603360036009001360236EC
:101196000336690E0024F66E6D0E0120F76E000E02
:1011A6000220F86E0900F5CF00F00900F5CF01F036
:1011B6000900F5CF02F00900F5CF03F092C204F062
:1011C60093C205F094C206F095C207F0D2EC04F083
:1011D60000C092F201C093F202C094F203C095F2ED
:1011E6000A0E046E91C200F07FDC08C000F000C059
:1011F60001F0000E00BEFF0E026E036E046E013695
:101206000190023603360436013601900236033663
:101216000436690E0124F66E6D0E0220F76E000E7E
:101226000320F86E0900F5CF00F00900F5CF01F0B4
:101236000900F5CF02F00900F5CF03F092C204F0E1
:1012460093C205F094C206F095C207F0D2EC04F002
:101256009DD0800E0A0A006E800E9119005C6FE226
:101266000A0E046E91C200F03FDC090E0024056EE2
:10127600000E00BEFF0E066E000E062205C000F030
:1012860006C001F0000E06BEFF0E026E036E0036AB
:1012960000900136023603360036009001360236DB
:1012A6000336690E0024F66E6D0E0120F76E000EF1
:1012B6000220F86E0900F5CF92F20900F5CF93F2FD
:1012C6000900F5CF94F20900F5CF95F20A0E046EE7
:1012D60091C200F009DC08C000F000C001F0000E69
:1012E60000BEFF0E026E036E046E013601900236DA
:1012F6000336043601360190023603360436690E8B
:101306000124F66E6D0E0220F76E000E0320F86EB5
:101316000900F5CF00F00900F5CF01F00900F5CF7F
:1013260002F00900F5CF03F092C204F093C205F073
:1013360094C206F095C207F0D2EC04F027D091C211
:1013460000F0000E91BFFF0E016E026E036E0036B6
:10135600009001360236033600360090013602361A
:101366000336690E0024F66E6D0E0120F76E000E30
:101376000220F86E0900F5CF00F00900F5CF01F064
:0E1386000900F5CF02F00900F5CF03F01200C8
:101394000B6A0A6A096A00500402F4CF09F0F3CF19
:1013A40008F001500502F4CF0BF0F3CF0AF000501F
:1013B4000502F3500926F4500A22E86A0B22015070
:1013C4000402F3500926F4500A22E86A0B2208C0EA
:1013D40000F009C001F00AC002F00BC003F01200D3
:1013E4000A6A0350D8A40A800750D8A40A820A5073
:1013F400D8B455EF0AF0030AD8B40EEF0AF00AB0D5
:1014040009EF0AF006AE53EF0AF051EF0AF002AE0C
:1014140051EF0AF053EF0AF00250800B0A6E029E5D
:101424000650800B069E0A18D8B41FEF0AF00A5023
:10143400D8B451EF0AF053EF0AF00750035CD8B464
:1014440029EF0AF0D8A045EF0AF04BEF0AF0065056
:10145400025CD8B433EF0AF0D8A045EF0AF04BEFA2
:101464000AF00550015CD8B43DEF0AF0D8A045EF6E
:101474000AF04BEF0AF00450005CD8B455EF0AF0C0
:10148400D8B04BEF0AF00A52D8B453EF0AF051EF38
:101494000AF00A52D8B451EF0AF053EF0AF0D88098
:0E14A4001200D8901200D880D88412001200D6
:0A14B200C582C5A201D0FDD71200CB
:1014BC000450000A12E10550000A0FE10650000A20
:1014CC000CE10750000A09E1FF0E006EFF0E016EE1
:1014DC007F0E026EFF0E036EA8D0086A096A0750D1
:1014EC00D8B409EF0BF00350D8B40EEF0BF0025048
:1014FC0006180A6E028E068E0E6A02C008F001C033
:10150C000CF000C00DF004500D5E0550D8A0053C49
:10151C000C5E0650D8A0063C085E086A0C6A0D6A80
:10152C00D8A0A0EF0AF0D890023201320032083273
:10153C00010E0E6E0750035ED8A0ADEF0AF07E0EC2
:10154C000E240326D8B013EF0BF0B3EF0AF07E0E87
:10155C000E240326D8A018EF0BF0180E0B6E0D36C8
:10156C000C3608360036013602360E360450005E54
:10157C000550D8A0053C015E0650D8A0063C025E82
:10158C0006340E120EA0CEEF0AF00D80D9EF0AF041
:10159C00045000260550D8B0053C01260650D8B0A2
:1015AC00062802260D900B2EB5EF0AF0FFEF0AF07D
:1015BC00D8900036013602360E360450005E0550C7
:1015CC00D8A0053C015E0650D8A0063C025E06344D
:1015DC000E10010B0D26D8B00C2AD8B4082AD8A4AA
:1015EC00FFEF0AF008320C320D32032AD8B413EF95
:1015FC000BF00AAE089E0850026E0C50016E0D5096
:10160C00006E1BEF0BF0010E65EC05F01BEF0BF001
:10161C00020E2FEC01F01BEF0BF0040E43EC01F06B
:0C162C001BEF0BF0080E36EC01F0120072
:101638000B6A0A6A096A086A0E6A03340836045093
:10164800085E0550D8A0053C095E0650D8A0063CA7
:101658000A5E0750D8A0073C0B5EE86AD8A0010EC6
:101668000E5E0336070E0C6E0334083609360A364A
:101678000B360E36045003A012D0085E0550D8A0D1
:10168800053C095E0650D8A0063C0A5E0750D8A063
:10169800073C0B5EE86AD8A0010E0E5E11D0082642
:1016A8000550D8B0053C09260650D8B0063C0A2695
:1016B8000750D8B0073C0B26E86AD8B0010E0E26B2
:1016C80003360C2ED1D70234083609360A360B36C3
:1016D8000E36045003A012D0085E0550D8A0053C71
:1016E800095E0650D8A0063C0A5E0750D8A0073C01
:1016F8000B5EE86AD8A0010E0E5E11D008260550D0
:10170800D8B0053C09260650D8B0063C0A26075032
:10171800D8B0073C0B26E86AD8B0010E0E26023670
:10172800070E0C6E0234083609360A360B360E36AA
:10173800045002A012D0085E0550D8A0053C095EEE
:101748000650D8A0063C0A5E0750D8A0073C0B5E9E
:10175800E86AD8A0010E0E5E11D008260550D8B050
:10176800053C09260650D8B0063C0A260750D8B0D2
:10177800073C0B26E86AD8B0010E0E2602360C2E5E
:10178800D1D70134083609360A360B360E360450DE
:1017980002A012D0085E0550D8A0053C095E06508C
:1017A800D8A0063C0A5E0750D8A0073C0B5EE86A42
:1017B800D8A0010E0E5E11D008260550D8B0053C01
:1017C80009260650D8B0063C0A260750D8B0073C70
:1017D8000B26E86AD8B0010E0E260136070E0C6EED
:1017E8000134083609360A360B360E36045001A085
:1017F80012D0085E0550D8A0053C095E0650D8A056
:10180800063C0A5E0750D8A0073C0B5EE86AD8A0E1
:10181800010E0E5E11D008260550D8B0053C0926E9
:101828000650D8B0063C0A260750D8B0073C0B260D
:10183800E86AD8B0010E0E2601360C2ED1D7003436
:10184800083609360A360B360E36045001A012D077
:10185800085E0550D8A0053C095E0650D8A0063C95
:101868000A5E0750D8A0073C0B5EE86AD8A0010EB4
:101878000E5E11D008260550D8B0053C0926065042
:10188800D8B0063C0A260750D8B0073C0B26E86AB1
:10189800D8B0010E0E260036070E0C6E003408363E
:1018A80009360A360B360E36045000A012D0085EF0
:1018B8000550D8A0053C095E0650D8A0063C0A5E33
:1018C8000750D8A0073C0B5EE86AD8A0010E0E5E50
:1018D80011D008260550D8B0053C09260650D8B0C6
:1018E800063C0A260750D8B0073C0B26E86AD8B051
:1018F800010E0E2600360C2ED1D700B00ED00450A3
:1019080008260550D8B0053C09260650D8B0063C34
:0C1918000A260750D8B0073C0B2612002E
:0E192400ACB202D00000FCD791C2ADFF1200A1
:101932000B6A0C6A0A6A086A0350D8B421EF0DF0E8
:10194200028E9E0E035E03BEACEF0CF0D8B4ACEF79
:101952000CF011EF0DF0036C080E035CD8A0DEEF63
:101962000CF0036E083600C008F001C000F002C09F
:1019720001F0026A080E035CD8A0DEEF0CF0036EE1
:10198200083600C008F001C000F0016A080E035CCE
:10199200D8A0DEEF0CF0036E083600C008F0006A33
:1019A200080E035CD8A0DEEF0CF0036E0836086A5E
:1019B2000350D8A4D890EAEF0CF00350D8B4EAEF61
:1019C2000CF0D8900232013200320832032EE2EFDC
:1019D2000CF00BBC08A0FBEF0CF0D8A0FBEF0CF056
:1019E200082AD8B4002AD8B4012AD8B4022A02BEDE
:1019F20025EF0DF00AAE21EF0DF0021E011E001EB2
:101A0200081E082AD8B4002AD8B4012AD8B4022A57
:101A120021EF0DF0026A016A006A086A21EF0DF0F7
:101A22000B800BAE2BEF0DF0026A0AAE2BEF0DF01E
:101A3200026E016E006E086E0A3602322BEF0DF056
:101A4200000E0C6A2CEF0DF0010E0C6E69EC05F025
:101A52002CEF0DF0FF0E0250036E0150026E00508B
:081A6200016E0850006E120035
:101A6A00F00E02019115006E0086008000C092F20D
:101A7A004FC196F2040E0010976F78EC02F000C086
:101A8A0065F1000E0101666F080E0D6E0D2EFED770
:101A9A004FC196F2FB0E02019215976F78EC02F095
:101AAA0000C065F1000E0101666F080E0D6E0D2E65
:101ABA00FED791C200F00036009000360090003642
:101ACA00009000360090F00E00160086008000C0DC
:101ADA0092F24FC196F2040E00100201976F78EC51
:101AEA0002F000C065F1000E0101666F080E0D6E6E
:101AFA000D2EFED74FC196F2FB0E02019215976F7B
:101B0A0078EC02F000C065F1000E0101666F080E64
:081B1A000D6E0D2EFED7120026
:101B22006E0E0201915DD8A0CAD0640E046E91C2FD
:101B320000F087EC02F0120E0024056E066A000E19
:101B4200062205C000F006C001F0000E06BEFF0E20
:101B5200026E036E003600900136023603360036FE
:101B62000090013602360336350E0024F66E6D0EF5
:101B72000120F76E000E0220F86E0900F5CF00F08A
:101B82000900F5CF01F00900F5CF02F00900F5CF09
:101B920003F0000E046E000E056E000E066E7E0E41
:101BA200076ED2EC04F000C092F201C093F202C0C0
:101BB20094F203C095F2640E046E91C200F087ECB9
:101BC20002F008C000F00A0E046E87EC02F0090E63
:101BD2000024056E066A000E062205C000F006C04B
:101BE20001F0000E06BEFF0E026E036E003600907C
:101BF20001360236033600360090013602360336CD
:101C0200350E0024F66E6D0E0120F76E000E0220D6
:101C1200F86E0900F5CF00F00900F5CF01F00900D8
:101C2200F5CF02F00900F5CF03F092C204F093C29F
:101C320005F094C206F095C207F0D2EC04F000C0A1
:101C420092F201C093F202C094F203C095F20A0E1E
:101C5200046E91C200F087EC02F008C000F000C0F0
:101C620001F0000E026E036E046E01360190023620
:101C72000336043601360190023603360436350E39
:101C82000124F66E6D0E0220F76E000E0320F86E30
:101C92000900F5CF00F00900F5CF01F00900F5CFFA
:101CA20002F00900F5CF03F092C204F093C205F0EE
:101CB20094C206F095C207F0D2EC04F0B1D0915173
:101CC2000A08D8B07ED00A0E046E91C200F087ECEA
:101CD20002F0090E0024056E066A000E062205C0F7
:101CE20000F006C001F0000E06BEFF0E026E036E8B
:101CF2000036009001360236033600360090013677
:101D020002360336350E0024F66E6D0E0120F76E94
:101D1200000E0220F86E0900F5CF00F00900F5CFA1
:101D220001F00900F5CF02F00900F5CF03F0000E33
:101D3200046E000E056E000E066E7E0E076ED2EC6D
:101D420004F000C092F201C093F202C094F203C008
:101D520095F20A0E046E91C200F087EC02F008C000
:101D620000F000C001F0000E026E036E046E013638
:101D720001900236033604360136019002360336EC
:101D82000436350E0124F66E6D0E0220F76E000E3B
:101D92000320F86E0900F5CF00F00900F5CF01F03D
:101DA2000900F5CF02F00900F5CF03F092C204F06A
:101DB20093C205F094C206F095C207F0D2EC04F08B
:101DC2002FD091C200F0000E016E026E036E00363B
:101DD2000090013602360336003600900136023694
:101DE2000336350E0024F66E6D0E0120F76E000EDE
:101DF2000220F86E0900F5CF00F00900F5CF01F0DE
:101E02000900F5CF02F00900F5CF03F0000E046ED1
:101E1200000E056E000E066E7E0E076ED2EC04F00A
:021E22001200AC
:101E24000050086E0150006E0250016E0350026EA5
:101E3400036A0B6A0C6A9E0E036E0A6A020E0C6E2B
:061E440066EC01F0120043
:081E4A00067EC2EC02F012005A
:101E520002016A6B695109081DE20A0E046E69C229
:101E620000F087EC02F000C06AF200C06AF26A3742
:101E72006A916A376A916A376A916A376A910A0E79
:101E8200046E69C200F087EC02F008C000F0005056
:0E1E92006A1302D069C26AF26AC200F012003E
:101EA000F00E02016915006E008600C06BF24FC192
:101EB00096F2040E0010976F78EC02F000C065F106
:101EC000000E0101666F100E0D6E0D2EFED7000084
:101ED0004FC196F2FB0E02016B15976F78EC02F082
:101EE00000C065F1000E0101666F100E0D6E0D2E23
:101EF000FED7000002016A5335E069C200F00036E7
:101F00000090003600900036009000360090F00EF1
:101F10000016008600C06BF24FC196F2040E00104E
:101F2000976F78EC02F000C065F1000E0101666F5A
:101F3000030E0D6E0D2EFED74FC196F2FB0E020161
:101F40006B15976F78EC02F000C065F1000E01018F
:101F5000666F210E0C6E760E0D6E0D2EFED70C2EBA
:061F6000FCD70000120096
:101F660002016C6B69C2E9FF6AC2EAFFEECF6BF24F
:101F76006B51000A0EE06BC291F2D1DC02016C2BB0
:101F86006C516925E96E000E6A21EA6EEECF6BF29E
:041F9600EFD712006F
:101F9A000C6A0E6A0250D8A4E6EF0FF001C002F0F4
:101FAA0000C001F0006A0E860250D8A4E6EF0FF0D6
:101FBA0001C002F0016A0E960E880250D8B4F8EFFA
:101FCA000FF00E50035ED8A4D8A0FEEF0FF0D89001
:101FDA0002BE04EF10F0003601360236032EEDEF92
:101FEA000FF0FEEF0FF0010E0C6E2FEC01F008EF70
:101FFA0010F0020E0C6E36EC01F008EF10F0040E31
:08200A000C6E4FEC01F0120016
:102012000D0E0201916F85DC0A0E0201916F81DCC7
:022022001200AA
:10202400086A096A100E0C6E013408360936045029
:10203400085E0550D8A0053C095ED8B007D004500E
:1020440008260550D8B0053C0926D890003601363C
:062054000C2EEAD7120079
:10205A0069C2F6FF6AC2F7FF6BC2F8FF0900F5CF43
:10206A0000F0005211E069C2F6FF6AC2F7FF6BC2C4
:10207A00F8FF0900F5CF91F2F3DC010E020169279E
:0A208A00000E6A236B23E4D7120056
:1020940057EC02F0D00E0201996F53EC01F069C2C3
:1020A40099F253EC01F059EC0AF0D10E0201996F48
:1020B40053EC01F00201916BE9EC05F000C06AF207
:0A20C40064EC01F06AC200F01200A3
:1020CE0002016B6B6C6B69C2E9FF6AC2EAFFEE50EC
:1020DE00000A16E0800E6C19006E800E005C02E1A4
:1020EE00140E6B5D0DE269C2E9FF6AC2EAFFEECF24
:1020FE0091F2B4DC0201694B6A2B6B4B6C2BE3D76C
:02210E001200BD
:1021100002016B6B6C6B0C0E026E69C200F06AC23E
:1021200001F0025005E001320032019EFF0FFAD7A4
:10213000E80E046E030E056ECAEC09F000C06BF2E7
:1021400001C06CF2000E6915036E6A510F0B046E2C
:1021500004C000F0016A640E046E000E056ECAEC45
:1021600009F000506B2701506C23F00E6915036EC7
:102170006AC204F0000E041603C000F004C001F0AF
:1021800001320032019E01320032019E01320032E2
:10219000019E01320032019E0A0E046E000E056E91
:1021A000CAEC09F000506B25026E01506C21036EE1
:1021B00002C06BF203C06CF20F0E6915006E6AC2AA
:1021C00001F0000E0116025000260350012200C04B
:0821D0006BF201C06CF2120079
:1021D8000201896B8A6B7D6B7E6B6BC200F06CC2EF
:1021E80001F06DC202F0010E6B27000E6C236D2307
:1021F80000C0F6FF01C0F7FF02C0F8FF0900F5CFE5
:1022080000F000C07AF20052D8B4FCEF20F07A5106
:10221800250A0BE069C2E1FF6AC2E2FF7AC2E6FF63
:10222800694B6A2B894B8A2BD8D77B6B7C6B7D6B70
:102238007E6B23D07D87010E6B27000E6C236D23E8
:1022480059D07D81010E6B27000E6C236D2352D06F
:102258007D83010E6B27000E6C236D234BD07E8788
:10226800010E6B27000E6C236D2344D07D85010E73
:102278006B27000E6C236D233DD06BC2F6FF6CC23A
:10228800F7FF6DC2F8FF0900F5CF01F001502D0AE4
:10229800D1E06BC2F6FF6CC2F7FF6DC2F8FF090010
:1022A800F5CF01F00150200ACCE06BC2F6FF6CC2FA
:1022B800F7FF6DC2F8FF0900F5CF01F001502B0AB6
:1022C800C7E06BC2F6FF6CC2F7FF6DC2F8FF0900EA
:1022D800F5CF01F00150230AC2E06BC2F6FF6CC2D1
:1022E800F7FF6DC2F8FF0900F5CF01F00150300A81
:1022F800BDE001D09ED77DA301D07D917DA701D0FF
:102308007D956BC2F6FF6CC2F7FF6DC2F8FF09003E
:10231800F5CF00F0000E016E00C091F2C6EC05F09A
:10232800005236E07B6B7C6B7BC200F07CC201F014
:102338000A0E046E000E056ECAEC09F06BC2F6FFB9
:102348006CC2F7FF6DC2F8FF0900F5CF02F002502A
:1023580000247B6F000E01207C6F300E7B5F000E27
:102368007C5B010E6B27000E6C236D236BC2F6FF9E
:102378006CC2F7FF6DC2F8FF0900F5CF00F0000E40
:10238800016E00C091F2C6EC05F00052CDE133D0E9
:102398006BC2F6FF6CC2F7FF6DC2F8FF0900F5CFFC
:1023A80001F001502A0A27E16EC2E9FF6FC2EAFF75
:1023B800EECF00F0EECF01F000C0E9FF01C0EAFF68
:1023C800EECF7BF2EECF7CF26EC2E9FF6FC2EAFF7E
:1023D800020EEE24006E000EEE20016E6EC2E1FFCA
:1023E8006FC2E2FF00C0E6FF01C0E6FF010E6B27E7
:1023F800000E6C236D236BC2F6FF6CC2F7FF6DC233
:10240800F8FF0900F5CF01F001502E0A70E1010E26
:102418006B27000E6C236D236BC2F6FF6CC2F7FFAF
:102428006DC2F8FF0900F5CF01F001502A0A28E132
:102438006EC2E9FF6FC2EAFFEECF00F0EECF01F007
:1024480000C0E9FF01C0EAFFEECF78F2EECF79F2E3
:102458006EC2E9FF6FC2EAFF020EEE24006E000EA4
:10246800EE20016E6EC2E1FF6FC2E2FF00C0E6FF20
:1024780001C0E6FF010E6B27000E6C236D2336D0DA
:10248800786B796B6BC2F6FF6CC2F7FF6DC2F8FF11
:102498000900F5CF00F0000E016E00C091F2C6EC05
:1024A80005F0005223E078C200F079C201F00A0E6C
:1024B800046E000E056ECAEC09F06BC2F6FF6CC222
:1024C800F7FF6DC2F8FF0900F5CF02F002500024B3
:1024D800786F000E0120796F300E785F000E795BFF
:1024E800010E6B27000E6C236D23CCD703D0786BBD
:1024F800796B7E896BC200F06CC201F06DC202F08C
:10250800010E6B27000E6C236D2300C0F6FF01C07F
:10251800F7FF02C0F8FF0900F5CF7AF2F9D089C2B7
:1025280000F08AC201F000EF21F07D89E3D77E85B3
:102538002ED17D8B7E812BD17E8329D17D8D27D194
:1025480026D17D8B7D8F23D16EC2E9FF6FC2EAFF52
:10255800EECF00F0EECF01F000C0E9FF01C0EAFFC6
:10256800EECF85F2EECF86F26EC2E9FF6FC2EAFFC8
:10257800020EEE24006E000EEE20016E6EC2E1FF28
:102588006FC2E2FF00C0E6FF01C0E6FF000E861939
:1025980002E1000E851904E1810E856F000E866F39
:1025A800876B886B87518525E96E88518621EA6E8D
:1025B800EE520BE0010E8725006E000E8821016E99
:1025C80000C087F201C088F2EDD7785179110AE08E
:1025D8008851795D02E18751785D04E278C287F21B
:1025E80079C288F27C51885D02E17B51875D05E202
:1025F80087517B5F88517C5B02D07B6B7C6B7DB79E
:1026080016D07BC200F07CC201F0010E7B5F000E89
:102618007C5B005001100BE069C2E1FF6AC2E2FF77
:10262800200EE66E694B6A2B894B8A2BEAD787C244
:1026380002F088C203F0010E875D006E000E885913
:10264800016E00C087F201C088F20250031019E041
:1026580085C2E9FF86C2EAFF69C2E1FF6AC2E2FFFA
:10266800EECFE6FF694B6A2B010E8525006E000E42
:102678008621016E00C085F201C086F2894B8A2B43
:10268800D6D77DA716D07BC200F07CC201F0010E20
:102698007B5F000E7C5B005001100BE069C2E1FF1C
:1026A8006AC2E2FF200EE66E694B6A2B894B8A2BC1
:1026B800EAD793D56EC2E9FF6FC2EAFFEECF00F00A
:1026C800EECF01F000C0E9FF01C0EAFFEECF7AF2D9
:1026D8006EC2E9FF6FC2EAFF020EEE24006E000E22
:1026E800EE20016E6EC2E1FF6FC2E2FF00C0E6FF9E
:1026F80001C0E6FF7A0E856F020E866F010E876FA6
:10270800000E886F62D7C00E7D13000E7E133FD077
:102718007A51000AD8B403D77A516C0AD8B405D7CD
:102728007A514C0AD8B401D77A51660AD8B4FFD680
:102738007A51450AD8B4FDD67A51650AD8B4FAD682
:102748007A51670AD8B4F8D67A516F0AD8B4F6D64F
:102758007A51640AD8B4F4D67A51690AD8B4F0D652
:102768007A51700AD8B4EDD67A51580AD8B4E9D655
:102778007A51780AD8B4E6D67A51730AD8B4E4D62E
:102788007A51630A97E07A51750ABDE0B3D7000E13
:102798007D15006E7E51070B016E00500110D8B4F4
:1027A800A3EF1CF07EA904D0060E786F000E796F97
:1027B8006EC2E9FF6FC2EAFFEECF00F0EECF01F084
:1027C80000C0E9FF01C0EAFFEECF7FF2EECF80F252
:1027D800EECF81F2EECF82F26EC2E9FF6FC2EAFF5E
:1027E800040EEE24006E000EEE20016E6EC2E1FFB4
:1027F8006FC2E2FF00C0E6FF01C0E6FF046A056A97
:10280800066A076A7FC200F080C201F081C202F046
:1028180082C203F0F2EC09F0010ED8B0000E006E8F
:10282800005205E0817F030E7D13000E7E13836B3B
:10283800846B7FC200F080C201F081C202F082C2C4
:1028480003F0046A056A066A076AD2EC05F0000E0E
:10285800D8A4010E006E0052D8B48AD082C200F00B
:10286800016A026A036AFF0E0016000E01167E0E48
:10287800005E000E015A00C083F201C084F2010E0E
:10288800005E000E015A00C083F201C084F2030EFC
:10289800046E000E056ECAEC09F000C083F201C098
:1028A80084F20A0E046E000E056E97EC06F000C066
:1028B80083F201C084F2800E0118026E800E025C61
:1028C80002E1000E005C05E2010E0201835F000ECA
:1028D800845B020183510008916FFBEC06F07FC214
:1028E80004F080C205F081C206F082C207F0D2EC83
:1028F80004F000C085F201C086F202C087F203C06E
:1029080088F2000E046E000E056E000E066E7F0E35
:10291800076E85C200F086C201F087C202F088C245
:1029280003F0F2EC09F0010ED8B0000E006E005270
:1029380005E0010E835F000E845B1AD0000E046E62
:10294800000E056E200E066E820E076E85C200F020
:1029580086C201F087C202F088C203F0F2EC09F0E7
:10296800000ED8B0010E006E005202E0834B842B9B
:10297800800E006E800E8419005C02E1835100080D
:1029880003E3010E7A6F02D083C27AF27EB118D0C7
:102998007EA315D0800E8419006E7F0E005C02E1C4
:1029A800FC0E835D0BE3800E8419006E800E79198E
:1029B800005C02E17851835D01E201D001D0F1D3DE
:1029C8007851791106E07EA304D0010E785F000EDD
:1029D800795B000E006E7951005C02E178510808BD
:1029E80003E2080E7A6F02D078C27AF27FC200F052
:1029F80080C201F081C202F082C203F0046A056A53
:102A0800066A076AD2EC05F0000ED8A4010E006E23
:102A18000052D8B44BD183C291F2FBEC06F000C04F
:102A280004F001C005F002C006F003C007F07FC241
:102A380000F080C201F081C202F082C203F05EECB5
:102A48000AF000C07FF201C080F202C081F203C028
:102A580082F202017A510008916FFBEC06F000C087
:102A680004F001C005F002C006F003C007F07FC201
:102A780000F080C201F081C202F082C203F05EEC75
:102A88000AF000C08BF201C08CF202C08DF203C0C4
:102A98008EF28BC27FF28CC280F28DC281F28EC21E
:102AA80082F28BC200F08CC201F08DC202F08EC29D
:102AB80003F099EC0CF012EC0FF000C004F001C028
:102AC80005F002C006F003C007F08BC200F08CC20C
:102AD80001F08DC202F08EC203F025EC0FF0000E5B
:102AE800046E000E056E000E066E7E0E076EF2EC8A
:102AF80009F0000ED8B0010E006E00521AE07FC235
:102B080000F080C201F081C202F082C203F0000E20
:102B1800046E000E056E000E066E7E0E076EC2EC89
:102B280002F000C07FF201C080F202C081F203C04F
:102B380082F27FC200F080C201F081C202F082C23C
:102B480003F099EC0CF002017A51010F096E0A6A40
:102B5800000E0A2209C004F00AC005F0000E0ABEE1
:102B6800FF0E066E076E04360490053606360736E5
:102B7800043604900536063607362B0E0424F66E06
:102B88006E0E0520F76E000E0620F86E0900F5CFD0
:102B980005F00900F5CF06F00900F5CF07F00900A8
:102BA800F5CF08F00850035C08E10750025C05E126
:102BB8000650015C02E10550005C1EE302017FC281
:102BC80000F080C201F081C202F082C203F0CD0E93
:102BD800046ECC0E056E4C0E066E7B0E076ED2ECA4
:102BE80004F000C07FF201C080F202C081F203C08D
:102BF80082F2834B842B5AD07FC200F080C201F04E
:102C080081C202F082C203F099EC0CF07AC204F09F
:102C1800000E056E066E076E0436049005360636FD
:102C28000736043604900536063607362B0E04247C
:102C3800F66E6E0E0520F76E000E0620F86E09007F
:102C4800F5CF05F00900F5CF06F00900F5CF07F03C
:102C58000900F5CF08F00850035C08E10750025C52
:102C680005E10650015C02E10550005C1FE202012B
:102C78007FC200F080C201F081C202F082C203F07C
:102C8800000E046E000E056E200E066E820E076E94
:102C9800D2EC04F000C07FF201C080F202C081F2E1
:102CA80003C082F2010E835F000E845B02017EA3E3
:102CB80093D07EB791D0800E000A006E800E7919ED
:102CC800005C02E178510A0804E20A0E786F000EEF
:102CD800796F7FC200F080C201F081C202F082C227
:102CE80003F099EC0CF000C085F201C086F202C036
:102CF80087F203C088F2855186118711881142E056
:102D08000A0E046E000E056E066E076E85C200F090
:102D180086C201F087C202F088C203F01CEC0BF0F7
:102D280008C000F009C001F00AC002F00BC003F0AF
:102D3800000E046E031808E10450021805E104505F
:102D4800011802E10050000A1DE1010E785F000E33
:102D5800795B0A0E046E000E056E066E076E85C25C
:102D680000F086C201F087C202F088C203F01CECB2
:102D78000BF000C085F201C086F202C087F203C0E2
:102D880088F2B9D7800E7919006E800E005C02E1D6
:102D98007A51785D21E278517A5D916FFBEC06F00B
:102DA80000C004F001C005F002C006F003C007F03F
:102DB8007FC200F080C201F081C202F082C203F03B
:102DC8005EEC0AF000C07FF201C080F202C081F21E
:102DD80003C082F278C27AF2050E02017825006EED
:102DE800000E7921016E00507B5F01507C5B7851A9
:102DF800791103E17EB701D004D0010E7B5F000E8C
:102E08007C5B030E7D15006E7EC201F0000E01167C
:102E18000050011004E0010E7B5F000E7C5B7DA575
:102E280039D07DA312D07DA103D02D0E706F02D0B2
:102E38002B0E706F69C2E1FF6AC2E2FF70C2E6FF43
:102E4800694B6A2B894B8A2B0CD07DA10AD069C2A9
:102E5800E1FF6AC2E2FF200EE66E694B6A2B894BDE
:102E68008A2B800E006E800E7C19005C02E17B517B
:102E780000080FE269C2E1FF6AC2E2FF300EE66EA7
:102E8800694B6A2B894B8A2B010E7B5F000E7C5B9A
:102E9800E8D73AD07DB718D0800E006E800E7C1926
:102EA800005C02E17B5100080FE269C2E1FF6AC2DF
:102EB800E2FF200EE66E694B6A2B894B8A2B010EC6
:102EC8007B5F000E7C5BE8D77DA312D07DA103D089
:102ED8002D0E716F02D02B0E716F69C2E1FF6AC2AD
:102EE800E2FF71C2E6FF694B6A2B894B8A2B0CD033
:102EF8007DA10AD069C2E1FF6AC2E2FF200EE66E38
:102F0800694B6A2B894B8A2B7FC200F080C201F083
:102F180081C202F082C203F099EC0CF000C085F285
:102F280001C086F202C087F203C088F27AC200F0BC
:102F3800000E016E026E036E0036009001360236F6
:102F48000336003600900136023603362B0E002475
:102F5800F66E6E0E0120F76E000E0220F86E090064
:102F6800F5CF04F00900F5CF05F00900F5CF06F01C
:102F78000900F5CF07F085C200F086C201F087C2CC
:102F880002F088C203F01CEC0BF0300E002669C278
:102F9800E1FF6AC2E2FF00C0E6FF694B6A2B894B7A
:102FA8008A2B7851791103E17EB701D06FD069C2BD
:102FB800E1FF6AC2E2FF2E0EE66E694B6A2B894B6F
:102FC8008A2B7A51785F000E795B7A534DE07A0745
:102FD8007AC200F0000E016E026E036E0036009099
:102FE80001360236033600360090013602360336C3
:102FF8002B0E0024F66E6E0E0120F76E000E0220D6
:10300800F86E0900F5CF04F00900F5CF05F00900C6
:10301800F5CF06F00900F5CF07F085C200F086C2AB
:1030280001F087C202F088C203F01CEC0BF00A0E14
:10303800046E000E056E066E076E1CEC0BF008C0E1
:1030480000F009C001F00AC002F00BC003F0300E16
:10305800002669C2E1FF6AC2E2FF00C0E6FF694BD1
:103068006A2B894B8A2BB1D7785179110FE069C245
:10307800E1FF6AC2E2FF300EE66E694B6A2B894BAC
:103088008A2B010E785F000E795BEED77DAB0BD0F3
:1030980069C2E1FF6AC2E2FF450EE66E694B6A2B20
:1030A800894B8A2B0AD069C2E1FF6AC2E2FF650E2A
:1030B800E66E694B6A2B894B8A2B800E8419006E49
:1030C800800E005C02E1000E835D11E2835100086E
:1030D800836F8451000E845769C2E1FF6AC2E2FF20
:1030E8002D0EE66E694B6A2B894B8A2B0AD069C272
:1030F800E1FF6AC2E2FF2B0EE66E694B6A2B894B31
:103108008A2B0A0E046E000E056E83C200F084C27C
:1031180001F097EC06F0300E002669C2E1FF6AC2A2
:10312800E2FF00C0E6FF0201694B6A2B894B8A2B3C
:103138000A0E046E000E056E83C200F084C201F010
:1031480097EC06F008C000F009C001F0300E002628
:1031580069C2E1FF6AC2E2FF00C0E6FF0201694BF3
:103168006A2B894B8A2B7DA71AD0800E006E800EA1
:103178007C19005C02E17B51000811E269C2E1FFA1
:103188006AC2E2FF200EE66E694B6A2B894B8A2BD6
:10319800010E7B5F000E7C5B7B517C11EFE1F1EF50
:1031A80010F07EA3F3D0800E8419006E800E005CB0
:1031B80002E1000E835D0AE2010E835D006E000EDF
:1031C8008459016E0050785F0150795B7FC200F02E
:1031D80080C201F081C202F082C203F099EC0CF0C7
:1031E80000C085F201C086F202C087F203C088F2EF
:1031F800010E7A6F7A510A0A34E07AC200F0000EA2
:10320800016E026E036E00360090013602360336F8
:10321800003600900136023603362B0E0024F66E77
:103228006E0E0120F76E000E0220F86E0900F5CF31
:1032380001F00900F5CF02F00900F5CF03F009000D
:10324800F5CF04F00450885D08E10350875D05E17F
:103258000250865D02E10150855D01E202D07A2BC1
:10326800C9D77A51785D8F6F000E7959906F8FC2E8
:1032780078F290C279F285C200F086C201F087C266
:1032880002F088C203F012EC0FF000C004F001C095
:1032980005F002C006F003C007F07FC200F080C24C
:1032A80001F081C202F082C203F025EC0FF000C0E9
:1032B8008BF201C08CF202C08DF203C08EF28FC275
:1032C80091F2FBEC06F08BC204F08CC205F08DC2C3
:1032D80006F08EC207F0D2EC04F0000E046E000E69
:1032E800056E000E066E7E0E076EC2EC02F099ECBB
:1032F8000CF000C085F201C086F202C087F203C05C
:1033080088F27851791142E00A0E046E000E056EBB
:10331800066E076E85C200F086C201F087C202F011
:1033280088C203F01CEC0BF008C000F009C001F0E3
:103338000AC002F00BC003F0000E046E031808E187
:103348000450021805E10450011802E10050000A77
:103358001DE10A0E046E000E056E066E076E85C22C
:1033680000F086C201F087C202F088C203F01CECAC
:103378000BF000C085F201C086F202C087F203C0DC
:1033880088F2010E785F000E795BBBD7800E006E65
:10339800800E7919005C02E178510C0816E378C2B6
:1033A80091F291EC0DF07FC204F080C205F081C269
:1033B80006F082C207F0C2EC02F000C07FF201C042
:1033C80080F202C081F203C082F27FC200F080C2A4
:1033D80001F081C202F082C203F0046A056A066A3B
:1033E800076AD2EC05F0000ED8A4010E006E005258
:1033F800D8B477D07FC200F080C201F081C202F059
:1034080082C203F099EC0CF0000E046E031808E178
:103418000450021805E10450011802E10050000AA6
:1034280060E1800E006E800E8419005C02E1835119
:10343800010857E283C291F2FBEC06F000C004F0E9
:1034480001C005F002C006F003C007F07FC200F01B
:1034580080C201F081C202F082C203F05EEC0AF081
:103468005F0E046E700E056E090E066E810E076EF5
:10347800F2EC09F0010ED8B0000E006E005206E022
:10348800090E0201835F000E845B05D00201080E5D
:10349800835F000E845B83C291F2FBEC06F000C0F0
:1034A80004F001C005F002C006F003C007F07FC2B7
:1034B80000F080C201F081C202F082C203F05EEC2B
:1034C8000AF099EC0CF000C085F201C086F202C047
:1034D80087F203C088F202017F6B806B816B826B7D
:1034E80038D07FC200F080C201F081C202F082C2EF
:1034F80003F099EC0CF000C085F201C086F202C01E
:1035080087F203C088F285C200F086C201F087C244
:1035180002F088C203F012EC0FF000C004F001C002
:1035280005F002C006F003C007F07FC200F080C2B9
:1035380001F081C202F082C203F025EC0FF000C056
:103548007FF201C080F202C081F203C082F2836B75
:10355800846B010E7A6F7A510A0A34E07AC200F05D
:10356800000E016E026E036E0036009001360236C0
:103578000336003600900136023603362B0E00243F
:10358800F66E6E0E0120F76E000E0220F86E09002E
:10359800F5CF01F00900F5CF02F00900F5CF03F0EF
:1035A8000900F5CF04F00450885D08E10350875DF9
:1035B80005E10250865D02E10150855D01E202D01D
:1035C8007A2BC9D77A517825006E000E7921016EC1
:1035D800835100268451012200507B5F01507C5B9F
:1035E8007EB704D07851791101E104D0010E7B5FD8
:1035F800000E7C5B030E7D15006E7EC201F0000E8E
:1036080001160050011004E0010E7B5F000E7C5B88
:103618007DA539D07DA312D07DA103D02D0E726F68
:1036280002D02B0E726F69C2E1FF6AC2E2FF72C25A
:10363800E6FF694B6A2B894B8A2B0CD07DA10AD0F7
:1036480069C2E1FF6AC2E2FF200EE66E694B6A2B8F
:10365800894B8A2B800E006E800E7C19005C02E17B
:103668007B5100080FE269C2E1FF6AC2E2FF300E37
:10367800E66E694B6A2B894B8A2B010E7B5F000E25
:103688007C5BE8D73AD07DB718D0800E006E800EEC
:103698007C19005C02E17B5100080FE269C2E1FF7E
:1036A8006AC2E2FF200EE66E694B6A2B894B8A2BB1
:1036B800010E7B5F000E7C5BE8D77DA312D07DA155
:1036C80003D02D0E736F02D02B0E736F69C2E1FF0A
:1036D8006AC2E2FF73C2E6FF694B6A2B894B8A2BE9
:1036E8000CD07DA10AD069C2E1FF6AC2E2FF200EB8
:1036F800E66E694B6A2B894B8A2B7AC200F07A07EF
:1037080000524CE07AC200F0000E016E026E036EA9
:103718000036009001360236033600360090013636
:10372800023603362B0E0024F66E6E0E0120F76E5D
:10373800000E0220F86E0900F5CF04F00900F5CF5D
:1037480005F00900F5CF06F00900F5CF07F085C2AE
:1037580000F086C201F087C202F088C203F01CECB8
:103768000BF00A0E046E000E056E066E076E1CEC5A
:103778000BF008C000F009C001F00AC002F00BC04D
:1037880003F0300E002669C2E1FF6AC2E2FF00C002
:10379800E6FF694B6A2B894B8A2BAFD7800E006EE8
:1037A800800E8419005C02E1835100080FE269C2AF
:1037B800E1FF6AC2E2FF300EE66E694B6A2B894B65
:1037C8008A2B010E835F000E845BE8D7800E000A07
:1037D800006E800E7919005C02E17851080803E256
:1037E800080E7A6F02D078C27AF27A51785F000EAA
:1037F800795B7A5303E17EB701D00AD069C2E1FF51
:103808006AC2E2FF2E0EE66E694B6A2B894B8A2B41
:103818007AC291F2FBEC06F07FC204F080C205F098
:1038280081C206F082C207F0D2EC04F0FFEC05F08A
:1038380000C085F201C086F202C087F203C088F298
:103848007A534DE07A077AC200F0000E016E026EDC
:10385800036E0036009001360236033600360090BB
:103868000136023603362B0E0024F66E6E0E01204A
:10387800F76E000E0220F86E0900F5CF04F009007B
:10388800F5CF05F00900F5CF06F00900F5CF07F0F0
:1038980085C200F086C201F087C202F088C203F038
:1038A8001CEC0BF00A0E046E000E056E066E076E19
:1038B8001CEC0BF008C000F009C001F00AC002F0CF
:1038C8000BC003F0300E002669C2E1FF6AC2E2FFB6
:1038D80000C0E6FF694B6A2B894B8A2BB1D7785118
:1038E80079110FE069C2E1FF6AC2E2FF300EE66EAD
:1038F800694B6A2B894B8A2B010E785F000E795B26
:10390800EED77DA71AD0800E006E800E7C19005C61
:1039180002E17B51000811E269C2E1FF6AC2E2FFDD
:10392800200EE66E694B6A2B894B8A2B010E7B5F52
:10393800000E7C5B7B517C11EFE1F1EF10F0C00EC3
:103948007D15016E7EC202F0000E0216000E0218EE
:1039580002E1000E0118D8A480D07DA927D06EC23C
:10396800E9FF6FC2EAFFEECF00F0EECF01F000C032
:10397800E9FF01C0EAFFEECF85F2EECF86F2EECF87
:1039880087F2EECF88F26EC2E9FF6FC2EAFF040E3B
:10399800EE24006E000EEE20016E6EC2E1FF6FC2D3
:1039A800E2FF00C0E6FF01C0E6FF2FD06EC2E9FFCC
:1039B8006FC2EAFFEECF00F0EECF01F000C0E9FFE2
:1039C80001C0EAFFEECF00F0EECF01F0000E01BE1D
:1039D800FF0E026E036E00C085F201C086F202C0BF
:1039E80087F203C088F26EC2E9FF6FC2EAFF020ED7
:1039F800EE24006E000EEE20016E6EC2E1FF6FC273
:103A0800E2FF00C0E6FF01C0E6FF800E8819006EE5
:103A1800800E005C08E1000E875D05E1000E865D02
:103A280002E1000E855D18E2030E7D13000E7E1381
:103A3800006A016A026A036A8551005E8651015A6A
:103A48008751025A8851035A00C085F201C086F294
:103A580002C087F203C088F24ED07DA927D06EC27B
:103A6800E9FF6FC2EAFFEECF00F0EECF01F000C031
:103A7800E9FF01C0EAFFEECF85F2EECF86F2EECF86
:103A880087F2EECF88F26EC2E9FF6FC2EAFF040E3A
:103A9800EE24006E000EEE20016E6EC2E1FF6FC2D2
:103AA800E2FF00C0E6FF01C0E6FF25D06EC2E9FFD5
:103AB8006FC2EAFFEECF00F0EECF01F000C0E9FFE1
:103AC80001C0EAFFEECF85F2EECF86F2000E876FD7
:103AD800886F6EC2E9FF6FC2EAFF020EEE24006E25
:103AE800000EEE20016E6EC2E1FF6FC2E2FF00C061
:103AF800E6FF01C0E6FF000E791902E1000E781911
:103B08000FE1000E006E881908E10050871905E1E1
:103B18000050861902E18551000A02E1784B792BA1
:103B2800C00E7D15006E00C005F0AED0010E7A6F94
:103B38007A510A0A34E07AC200F0000E016E026E71
:103B4800036E0036009001360236033600360090C8
:103B58000136023603362B0E0024F66E6E0E012057
:103B6800F76E000E0220F86E0900F5CF01F009008B
:103B7800F5CF02F00900F5CF03F00900F5CF04F006
:103B88000450885D08E10350875D05E10250865DB9
:103B980002E10150855D01E202D07A2BC9D782D0BB
:103BA800010E7A6F7A51080A34E07AC200F0000EEA
:103BB800016E026E036E003600900136023603363F
:103BC80000360090013602360336960E0024F66E53
:103BD8006E0E0120F76E000E0220F86E0900F5CF78
:103BE80001F00900F5CF02F00900F5CF03F0090054
:103BF800F5CF04F00450885D08E10350875D05E1C6
:103C08000250865D02E10150855D01E202D07A2B07
:103C1800C9D748D0010E7A6F7A510C0A34E07AC2BB
:103C280000F0000E016E026E036E00360090013641
:103C38000236033600360090013602360336D00EBF
:103C48000024F66E6D0E0120F76E000E0220F86E4D
:103C58000900F5CF01F00900F5CF02F00900F5CF12
:103C680003F00900F5CF04F00450885D08E1035023
:103C7800875D05E10250865D02E10150855D01E244
:103C880002D07A2BC9D70ED00550000AD8B44ED727
:103C98000550C00AD8B44AD70550800A81E00550BB
:103CA800400AB8E0800E006E800E7919005C02E1CF
:103CB80078517A5D03E278C27AF20DD0800E7919D4
:103CC800006E800E005C02E17A51785D04E27AC2EF
:103CD80078F2000E796F7B517C110EE0030E7D1592
:103CE800006E7EC201F0000E01160050011004E0C3
:103CF800010E7B5F000E7C5B800E7919006E800ED2
:103D08007C19005C02E17B51785D05E278517B5FAC
:103D180079517C5B02D07B6B7C6BC40E7D15016E88
:103D28007E51080B026E0250080A02E1400E01188B
:103D380008E17B517C1104E0010E7B5F000E7C5B87
:103D48001CD0C00E7D15016E7E51080B026E02500C
:103D5800080A02E1800E011810E1800E006E800E44
:103D68007C19005C02E17B51020805E2020E7B5FD0
:103D7800000E7C5B02D07B6B7C6B7DA55DD07DA348
:103D880012D07DA103D02D0E746F02D02B0E746F4C
:103D980069C2E1FF6AC2E2FF74C2E6FF694B6A2B9F
:103DA800894B8A2B34D07DA10BD069C2E1FF6AC24E
:103DB800E2FF200EE66E694B6A2B894B8A2B27D0CF
:103DC800C00E7D15016E7E51080B026E0250080A66
:103DD80002E1800E01181BE169C2E1FF6AC2E2FF3D
:103DE800300EE66E694B6A2B894B8A2B7DAB03D06C
:103DF800580E756F02D0780E756F69C2E1FF6AC2FE
:103E0800E2FF75C2E6FF694B6A2B894B8A2B7B510F
:103E18007C1111E069C2E1FF6AC2E2FF300EE66E72
:103E2800694B6A2B894B8A2B010E7B5F000E7C5BEA
:103E38007B517C11EFE174D07B517C1113E07DB78D
:103E480011D069C2E1FF6AC2E2FF200EE66E694B3B
:103E58006A2B894B8A2B010E7B5F000E7C5B7B51A2
:103E68007C11EFE17DA312D07DA103D02D0E766FDA
:103E780002D02B0E766F69C2E1FF6AC2E2FF76C2FA
:103E8800E6FF694B6A2B894B8A2B0CD07DA10AD09F
:103E980069C2E1FF6AC2E2FF200EE66E694B6A2B37
:103EA800894B8A2BC00E7D15016E7E51080B026E60
:103EB8000250080A02E1400E01180BE169C2E1FF55
:103EC8006AC2E2FF300EE66E694B6A2B894B8A2B79
:103ED80027D0C00E7D15016E7E51080B026E025070
:103EE800080A02E1800E01181BE169C2E1FF6AC2FB
:103EF800E2FF300EE66E694B6A2B894B8A2B7DAB4D
:103F080003D0580E776F02D0780E776F69C2E1FF41
:103F18006AC2E2FF77C2E6FF694B6A2B894B8A2B9C
:103F2800800E006E800E7919005C02E178517A5D8E
:103F38000BE269C2E1FF6AC2E2FF300EE66E694B2E
:103F48006A2B894B8A2BECD778C200F079C201F032
:103F5800010E785F000E795B00500110D8B42AD1A9
:103F6800C00E7D15006E00C08BF20AD178C200F039
:103F780079C201F0000E79BFFF0E026E036E0036A3
:103F880000900136023603360036009001360236BC
:103F980003362B0E0024F66E6E0E0120F76E000E0F
:103FA8000220F86E0900F5CF04F00900F5CF05F0FE
:103FB8000900F5CF06F00900F5CF07F085C200F03B
:103FC80086C201F087C202F088C203F01CEC0BF035
:103FD8000A0E046E000E056E066E076E1CEC0BF0E2
:103FE80008C000F009C001F00AC002F00BC003F0DD
:103FF800300E00247A6FD3D07DAB45D078C200F064
:1040080079C201F0000E79BFFF0E026E036E003612
:10401800009001360236033600360090013602362B
:104028000336960E0024F66E6E0E0120F76E000E13
:104038000220F86E0900F5CF04F00900F5CF05F06D
:104048000900F5CF06F00900F5CF07F085C200F0AA
:1040580086C201F087C202F088C203F01CEC0BF0A4
:104068000F0E0016000E011602160316430E00244A
:10407800F66E700E0120F76E000E0220F86E090031
:10408800F5CF7AF244D078C200F079C201F0000E80
:1040980079BFFF0E026E036E0036009001360236BD
:1040A800033600360090013602360336960E002499
:1040B800F66E6E0E0120F76E000E0220F86E0900F3
:1040C800F5CF04F00900F5CF05F00900F5CF06F0AB
:1040D8000900F5CF07F085C200F086C201F087C25B
:1040E80002F088C203F01CEC0BF00F0E0016000E55
:1040F800011602160316540E0024F66E700E0120E7
:10410800F76E000E0220F86E0900F5CF7AF247D05C
:1041180078C200F079C201F0000E79BFFF0E026E7E
:10412800036E0036009001360236033600360090E2
:10413800013602360336D00E0024F66E6D0E0120CD
:10414800F76E000E0220F86E0900F5CF04F00900A2
:10415800F5CF05F00900F5CF06F00900F5CF07F017
:1041680085C200F086C201F087C202F088C203F05F
:104178001CEC0BF0070E00147A6F300E7A270FD064
:104188008B51000AD8B4F2D68B51C00AD8B4EED6F7
:104198008B51800AD8B430D78B51400AB9E069C234
:1041A800E1FF6AC2E2FF7AC2E6FF694B6A2B894BDC
:1041B8008A2BCAD67DA71AD0800E006E800E7C1975
:1041C800005C02E17B51000811E269C2E1FF6AC2AA
:1041D800E2FF200EE66E694B6A2B894B8A2B010E93
:1041E8007B5F000E7C5B7B517C11EFE1F1EF10F0FF
:0A41F80089C200F08AC201F0120033
:104202000201586B050E585D0AE258515625E16EBF
:10421200000E5721E26E200EE66E582BF3D758514E
:104222005625E16E000E5721E26EE66A5807585194
:104232005625596F000E57215A6F0A0E046E000E52
:10424200056E54C200F055C201F012EC10F008C025
:1042520000F009C001F0300E002659C2E1FF5AC237
:10426200E2FF00C0E6FF0A0E046E000E056E54C2A5
:1042720000F055C201F012EC10F000C054F201C07F
:1042820055F2000E011802E1000E001801E102D001
:064292005807CDD7120011
:1042980058C201F059C202F0010E0201585F000E27
:1042A800595B000E021802E1000E01181FE054C20B
:1042B800E9FF55C2EAFF56C2D9FF57C2DAFFEE50EE
:1042C800DE180FE054C2E9FF55C2EAFF56C2D9FF13
:1042D80057C2DAFFDE50EE5C006E016A000E015A2A
:1042E80007D0544B552B564B572BD2D7006A016A2F
:0242F8001200B2
:1042FA000101D46BD26BD36BCA6BCB6BD06BD16B16
:10430A000201316B326B016A026A800E0218006E7A
:10431A00800E005C02E1200E015C0AE2D40E012448
:10432A00E16E010E0220E26EE66A014A022AEDD728
:0C433A00AECF01F0000E026E9D8A120052
:10434600A69C54C2A9FFA69EA680A8CF00F0120084
:1043560054C2F6FF55C2F7FF56C2F8FF0900F5CF63
:1043660000F0005212E054C2F6FF55C2F7FF56C2E3
:10437600F8FF0900F5CF91F292EC0CF0010E020164
:0C4386005427000E55235623E3D71200E5
:10439200590E0201676F020E686F54C269F255C26C
:1043A2006AF256C26BF257C26CF258C26DF2670ED5
:1043B2006E6F020E6F6FECEC10F000C065F201C080
:1043C20066F200505425E16E01505521E26EE66A14
:0A43D20065C200F066C201F012009F
:1043DC0056C2F6FF57C2F7FF58C2F8FF0900F5CFD7
:1043EC0000F0005218E056C2F6FF57C2F7FF58C251
:1043FC00F8FF0900F5CF00F054C2E1FF55C2E2FF0F
:10440C0000C0E6FF0201544B552B010E5627000E3F
:10441C0057235823DDD754C2E1FF55C2E2FFE66AA9
:02442C0012007C
:10442E0000C008F00150006E016A026A036A0B6A4E
:10443E000C6A016A026A036A960E036E0A6A00AE7D
:10444E002FEF22F0081E001E082AD8B4002A0A8E6A
:10445E0000C001F008C000F0086A026ACDEC0FF04F
:02446E0012003A
:104470000201696B4AEC10F000C05CF1010E020110
:10448000696F4AEC10F000C0CCF1020E0201696FB6
:104490004AEC10F000C0CDF1030E0201696F4AEC46
:1044A00010F000C0C9F1040E0201696F4AEC10F06F
:1044B00000C0C8F1050E0201696F4AEC10F000C09F
:1044C000C7F1060E0201696F4AEC10F000C0C6F198
:1044D000CDC156F202015633569F5633569F56337E
:1044E000569F5633569F030E696F29EC0FF000500C
:1044F00056150001786F300E78270F0E0101CD158B
:104500000001796F300E7927CCC156F20201563383
:10451000569F5633569F5633569F5633569F070E17
:10452000696F29EC0FF00050561500017B6F300EBB
:104530007B270F0E0101CC1500017C6F300E7C270C
:104540005CC156F202015633569F5633569F56337E
:10455000569F5633569F070E696F29EC0FF0005097
:10456000561500017E6F300E7E270F0E01015C157F
:1045700000017F6F300E7F27C8C156F2020156330B
:10458000569F5633569F5633569F5633569F070EA7
:10459000696F29EC0FF00050561500016F6F300E57
:1045A0006F270F0E0101C8150001706F300E7027C4
:1045B000C7C156F202015633569F5633569F5633A3
:1045C000569F5633569F070E696F29EC0FF0005027
:1045D00056150001726F300E72270F0E0101C715BC
:1045E0000001736F300E7327C6C156F202015633B5
:1045F000569F5633569F5633569F5633569F070E37
:10460000696F29EC0FF0005056150001756F300EE0
:1046100075270F0E0101C6150001766F300E762743
:10462000CDC169F2000E02016A6F88EC10F0100E25
:10463000046E0E0E056ECAEC09F000C056F201C001
:1046400057F2CCC169F2000E6A6F88EC10F03C0E94
:10465000046E000E056ECAEC09F00050562701509A
:1046600057235CC169F2000E6A6F88EC10F00050AD
:1046700056250101556F0150020157210101566F66
:10468000000E576F586F010E02015415016E55C28E
:1046900002F0000E0216000E021802E1010E0118CF
:1046A0005BE1800E696F010E6A6F50EC0FF0820EB5
:1046B0000C6EDD0E0D6E0D2EFED70C2EFCD70000FD
:1046C0000000010159A718D0FE0E0201696F700E9B
:1046D0006A6F000E6B6F2DEC10F0860E0201696F91
:1046E000010E6A6F50EC0FF0780E0201696F000E38
:1046F0006A6F67EC10F030D00201F70E696F700E30
:104700006A6F000E6B6F2DEC10F0860E0201696F60
:10471000010E6A6F50EC0FF06F0E0201696F000E10
:104720006A6F67EC10F08F0E696F010E6A6F50ECC4
:104730000FF0060E006E000E016EC9C104F0000EEF
:10474000056ECAEC09F0260E00240201696F000E06
:1047500001206A6F67EC10F0020E5415016E55C20D
:1047600002F0000E0216000E021802E1020E0118FD
:104770002AE1060E006E000E016EC9C104F0000EA3
:10478000056ECAEC09F0260E0024696F000E0120A8
:104790006A6FB3EC0FF0090E916F92EC0CF06F0E94
:1047A0000201696F000E6A6FB3EC0FF0090E916F92
:1047B00092EC0CF0780E0201696F000E6A6FB3EC98
:0847C0000FF009EC10F01200EB
:1047C8000B6A0350D8B42AEF24F002500A6E028E06
:1047D8008E0E035E03AE2EEF24F0036C080E035C0E
:1047E800D8A009EF24F0036E013602C001F0026A76
:1047F800080E035CD8A009EF24F0036E0136016AA5
:104808000350D8A4D89013EF24F00350D8B413EF72
:1048180024F0D89002320132032E0DEF24F00BBCA5
:1048280001A020EF24F0D8A020EF24F0012AD8B46A
:10483800022A02BE3DEF24F00AAE43EF24F0021E26
:10484800011E012AD8B4022A43EF24F0026A016A41
:1048580043EF24F00B800BAE47EF24F0026A0AAE58
:1048680047EF24F0FF0E026E016E0A36023247EF60
:1048780024F0010E0C6E69EC05F049EF24F0000EEF
:104888000C6E49EF24F0FF0E0C6E0150006E0250C2
:04489800016E12009B
:10489C0054C2E9FF55C2EAFFEECF56F2000E0201F8
:1048AC00576F000E576F000E571902E1200E561964
:1048BC0007E0000E571902E1090E561901E003D06A
:1048CC00544B552BE5D7586B596B5A6B5B6B000EE1
:1048DC00571902E12D0E561905E15A4B5B2B544B1F
:1048EC00552B08D0000E571902E12B0E561902E178
:1048FC00544B552B54C2E9FF55C2EAFFEECF56F28A
:10490C00000E576F000E576F56C291F2C6EC05F0B1
:10491C00005219E058C200F059C201F00A0E046EA0
:10492C00000E056ECAEC09F0300E565D026E000EDC
:10493C005759036E02500024586F03500120596FD1
:10494C00544B552BD7D75A515B1108E058510008DE
:10495C00006E59C201F0000E015604D058C200F08E
:06496C0059C201F0120027
:10497200A6A202D00000FCD7A69C54C2A9FF55C231
:10498200A8FFA69EA684F2CF00F0F29E550EA76E57
:10499200AA0EA76EA68200BE02D0F29E01D0F28EAF
:0449A200A6941200C5
:1049A60057EC02F0D00E0201996F53EC01F054C29D
:1049B60099F253EC01F055C299F253EC01F064EC14
:0449C60001F01200EA
:1049CA0054C204F055C205F002015851591124E0AD
:1049DA00010E585F000E595B04C002F005C003F0D7
:1049EA00044A052A56C200F057C201F0564B572B0B
:1049FA0000C0E9FF01C0EAFF02C0E1FF03C0E2FF15
:104A0A00EECFE6FF02C0E9FF03C0EAFFEECF00F0F7
:104A1A00005201E101D0D8D758C200F059C201F0C2
:104A2A00010E585F000E595B0050011008E004C0E7
:104A3A00E1FF05C0E2FFE66A044A052AEDD754C23F
:084A4A0000F055C201F012005A
:104A5200FF0E816E8F0E936E938093829384938662
:104A6200070E806E2F0E926E840EC16EC196C184A7
:104A7200C192C190800E826EFF0E946E94869488CD
:084A8200948E949C94921200A2
:104A8A0002013C6B3D6B39C2F6FF3AC2F7FF3BC2EB
:104A9A00F8FF0900F5CF01F00150000A1DE0800E71
:104AAA003D19006E800E005C02E1140E3C5D14E2BA
:104ABA0039C2F6FF3AC2F7FF3BC2F8FF0900F5CF49
:104ACA0091F235EC0DF0010E02013927000E3A235E
:0A4ADA003B233C4B3D2BD7D71200C5
:104AE400F2AE03D0010E02013D6FF29E060E006E7F
:104AF40039C23BF23AC23CF2005006E002013B37B5
:104B04003B913C37FF0FF9D70201FF0E3B177F0E95
:104B14003C1722EC01F057EC02F0A20E0201996F4F
:104B240053EC01F000C088F03CC299F253EC01F060
:104B340000C088F03BC299F253EC01F000C088F049
:104B440059EC0AF0A30E0201996F53EC01F000C076
:104B540088F022EC01F002013B6B3C6B000E3C5DE3
:104B640002E13F0E3B5D14E2AB0E3B253E6F000EAF
:104B74003C213F6F010E916FE9EC05F03EC2E1FF6D
:104B84003FC2E2FF00C0E6FF02013B4B3C2BE6D7ED
:104B9400AB0E3B253E6F000E3C213F6F916BE9EC61
:104BA40005F03EC2E1FF3FC2E2FF00C0E6FF64EC55
:104BB40001F022EC01F002013D51010AD8B4F28E59
:024BC4001200DD
:104BC60039C23AF2000E02013B6F3AC254F2A3EC2C
:104BD60021F000C03CF2000E3D6F000E3D1902E1CF
:104BE600000E3C1901E12ED0800E006E800E3B199E
:104BF600005C02E13A51FE0801E224D03CC291F287
:104C060092EC0CF0020139513A5D006E000E3B59F0
:104C1600016E890E0024E16E000E0120E26E3CC298
:104C2600E6FF210E0C6E760E0D6E0D2EFED70C2EA7
:104C3600FCD700003A4B3B2B000E3D1902E1000E5B
:064C46003C19C3E112005D
:104C4C000900F5CFE6FF0006FBE10106F9E11200D1
:104C5C00240E0101966F190E976F910E986F020E2C
:104C6C00996FB40E9A6F4C0E9B6F000E9C6F000EDA
:104C7C009D6FFF0E926FFF0E936F000E946F000EE0
:104C8C00956FFF0E8C6FFF0E8D6F000E8E6F000EEA
:104C9C008F6FAC8A900EAB6E948E949C9EAA03D0B0
:084CAC00AECF00F0FBD71200AF
:104CB400AECF01F0ABA202D0AB98AB8801C000F03C
:024CC4001200DC
:104CC600949894968B988B9694889486C79EC79C46
:064CD600380EC66E12004C
:104CDC00CD6ACD8ACD880B0ECF6EDB0ECE6E020167
:104CEC00336B346B0101C46BC56B9E909D90CD9062
:024CFC001200A4
:104CFE00FE0E0201546FA3EC21F000C08BF100C038
:104D0E0039F2000E3A6FFF0E546FA3EC21F000C083
:104D1E008BF139C254F10101536B00505327000E31
:104D2E005423880E0201546F6C0E556F000E566F91
:104D3E00ABEC21F0EB0E0101CE6F000ECF6F53C125
:104D4E0054F254C155F2CEC156F2CFC157F201EC16
:104D5E0021F0CEC169F2CFC16AF2B3EC0FF009ECCB
:0A4D6E0010F00101516B526B1200AE
:104D7800F2AE03D0010E02013D6FF29E0001A96B55
:104D8800AA6B060E006E39C23BF23AC23CF20050E2
:104D980006E002013B373B913C37FF0FF9D7020190
:104DA800FF0E3B177F0E3C1722EC01F057EC02F088
:104DB800A20E0201996F53EC01F000C088F03CC2CA
:104DC80099F253EC01F000C088F03BC299F253EC21
:104DD80001F000C088F00050000803E20001A94B70
:104DE800AA2B02013B6B3C6B000E3C5D02E1400EBE
:104DF8003B5D16E2AB0E3B25E96E000E3C21EA6EE8
:104E0800EECF99F253EC01F000C088F00050000892
:104E180003E20001A94BAA2B02013B4B3C2BE4D730
:104E280064EC01F022EC01F002013D51010AD8B412
:044E3800F28E1200E4
:104E3C000101516B526B54C100F0016AFE0E02016C
:104E4C00546F00C055F28FDD820E0C6EDD0E0D6EB0
:104E5C000D2EFED70C2EFCD700000000FF0E01011A
:104E6C0053150201556FFF0E546F7DDD820E0C6ED3
:104E7C00DD0E0D6E0D2EFED70C2EFCD700000000A3
:024E8C00120012
:104E8E00020E0201396F000E3A6F0101D26BD36B25
:104E9E009D9A800ED119006E800E005C02E1150EF7
:104EAE00D05DD8B0CED0CEC154F2CFC155F2530E94
:104EBE000201566F6E0E576F000E586FD40E596F5B
:104ECE00010E5A6FD0C15BF2D1C15CF2C9EC21F078
:104EDE00CEC191F292EC0CF0020E02012F6F000E79
:104EEE00306F800E3019006E800E0101D119005CFA
:104EFE0003E1D05102012F5D37E20201D40E2F25BE
:104F0E00E96E010E3021EA6EEECF01F001503B0A40
:104F1E0027E1D40E2F25E16E010E3021E26EE66AF6
:104F2E00260E0101D22502013B6F020E0101D32193
:104F3E0002013C6FD40E3925546F010E3A21556F84
:104F4E00A6DC3BC2E1FF3CC2E2FF00C0E6FF010E61
:104F5E002F25396F000E30213A6F0101D24BD32B22
:104F6E0002012F4B302BBDD70201010E245D006EC6
:104F7E00000E2559016ED40E0024E16E010E0120A3
:104F8E00E26EE66A260E0101D22502013B6F020E89
:104F9E000101D32102013C6FD40E3925546F010E4D
:104FAE003A21556F74DC3BC2E1FF3CC2E2FF00C008
:104FBE00E6FF26C2C8F127C2C7F128C2C6F129C230
:104FCE00C9F12AC2CDF12BC2CCF1546B500E556FE4
:104FDE00E3DCCCC169F229EC0FF000C055F2010EF2
:104FEE00546FDADCCDC169F229EC0FF000C055F236
:104FFE00020E546FD1DCC9C169F229EC0FF000C06A
:10500E0055F2030E546FC8DCC8C169F229EC0FF0DB
:10501E0000C055F2040E546FBFDCC7C169F229EC13
:10502E000FF000C055F2050E546FB6DCC6C169F222
:10503E0029EC0FF000C055F2060E546FADDC7DEC7E
:06504E0021F09D8A120012
:1050540039C244F23AC245F23BC246F23CC247F27C
:1050640002013F51000805E3070E406F000E416F37
:1050740012D03F51160805E2170E426F000E436F1F
:1050840006D03F51010F426F436B000E432342C2CF
:1050940040F243C241F240C24EF241C24FF2486B69
:1050A400496B046A056A066A076A44C200F045C28D
:1050B40001F046C202F047C203F0F2EC09F0010E1F
:1050C400D8B0000E006E005209E03DC2E1FF3EC2BE
:1050D400E2FF2D0EE66E3D4B3E2B467F44C204F0AC
:1050E40045C205F046C206F047C207F0006A016AED
:1050F400026A036AF2EC09F0010ED8B0000E006EE9
:10510400005237E0000E046E000E056E000E066EAF
:105114007F0E076E44C200F045C201F046C202F0A1
:1051240047C203F0F2EC09F0010ED8B0000E006E95
:1051340000521FE044C200F045C201F046C202F032
:1051440047C203F0000E046E000E056E200E066EBC
:10515400820E076ED2EC04F000C044F201C045F2A6
:1051640002C046F203C047F2010E485F000E495BDD
:10517400C9D7000E046E000E056E200E066E820E58
:10518400076E44C200F045C201F046C202F047C2B5
:1051940003F0F2EC09F0000ED8B0010E006E0052DC
:1051A4001EE0000E046E000E056E200E066E820ECA
:1051B400076E44C200F045C201F046C202F047C285
:1051C40003F05EEC0AF000C044F201C045F202C0F4
:1051D40046F203C047F20201484B492BCAD7485153
:1051E4004E2749514F23010E4A6F000E4B6F010E9B
:1051F400006E000E016E17EC22F000C050F201C0E8
:1052040051F202C052F203C053F2800E4B19006EE9
:10521400800E4F19005C02E14E514A5D1EE2000E01
:10522400046E000E056E200E066E820E076E50C2CE
:1052340000F051C201F052C202F053C203F05EEC1E
:105244000AF000C050F201C051F202C052F203C091
:1052540053F202014A4B4B2BD8D7000E046E000EBA
:10526400056E000E066E800E076E50C200F051C22D
:1052740001F052C202F053C203F05EEC0AF044C2E1
:1052840004F045C205F046C206F047C207F0C2EC7E
:1052940002F000C044F201C045F202C046F203C06D
:1052A40047F2000E046E000E056E200E066E820E8E
:1052B400076EF2EC09F0000ED8B0010E006E005239
:1052C4000BE0000E0201446F000E456F000E466FA6
:1052D4007F0E476F484B492B0201800E4919006E1F
:1052E400800E005C02E1000E485D38E23DC2E1FF41
:1052F4003EC2E2FF300EE66E3D4B3E2B3DC2E1FF67
:105304003EC2E2FF2E0EE66E3D4B3E2B800E4F1941
:10531400006E800E005C02E1000E4E5D04E24E5110
:10532400485F4F51495BFF0E4A6FFF0E4B6F800E73
:105334004919006E800E4B19005C02E14A51485D28
:105344000DE23DC2E1FF3EC2E2FF300EE66E3D4B90
:105354003E2B010E4A5F000E4B5BE9D74A6B4B6B49
:10536400800E4B19006E800E4F19005C02E14E5105
:105374004A5D63E244C200F045C201F046C202F055
:1053840047C203F0E4EC23F000C04CF201C04DF23C
:10539400300E00263DC2E1FF3EC2E2FF00C0E6FF40
:1053A4003D4B3E2B4B51491902E148514A1908E142
:1053B4003DC2E1FF3EC2E2FF2E0EE66E3D4B3E2BA8
:1053C4004CC200F04DC201F017EC22F000C050F2C4
:1053D40001C051F202C052F203C053F200C004F003
:1053E40001C005F002C006F003C007F044C200F09B
:1053F40045C201F046C202F047C203F025EC0FF0AB
:1054040000C044F201C045F202C046F203C047F2B4
:10541400000E046E000E056E200E066E820E076EE0
:10542400D2EC04F000C044F201C045F202C046F2DE
:1054340003C047F24A4B4B2B93D73DC2E1FF3EC218
:06544400E2FFE66A12001F
:10544A000201396B3A6B800E3A19006E800E005CCD
:10545A0002E1400E395D0AE2AB0E3925E16E000E1B
:10546A003A21E26EE66A394B3A2BEDD7010E546FB8
:10547A00000E556F38EC22F00101516B526BAB0EE6
:10548A0051250201546F000E010152210201556F8C
:10549A006F0E566F000E576F050E586F000E596F3C
:1054AA00E5EC24F0050E0101516F000E526FAB0EB0
:1054BA005125E16E000E5221E26E3B0EE66E060E9B
:1054CA00516F000E526FAB0E51250201546F000E40
:1054DA00010152210201556F780E566F000E576F67
:1054EA00050E586F000E596FE5EC24F00B0E010102
:1054FA00516F000E526FAB0E5125E16E000E522114
:10550A00E26E3B0EE66E0C0E516F000E526F0001FA
:10551A00B76BEB0E0101CE6F000ECF6FCEC154F206
:10552A00CFC155F29D0E0201566F6D0E576F000ED8
:10553A00586FAB0E596F000E5A6F0C0E5B6F000E50
:10554A005C6FC9EC21F0CEC169F2CFC16AF2B3EC4B
:04555A000FF012003C
:10555E0002013F6B406B000E405D02E10A0E3F5DA3
:10556E000BE23F513D25E16E40513E21E26E200E91
:10557E00E66E3F4B402BEFD73F513D25E16E40513C
:10558E003E21E26EE66A010E3F5F000E405B3F5128
:10559E003D25416F40513E21426F0A0E046E000EB2
:1055AE00056E066E076E39C200F03AC201F03BC2BC
:1055BE0002F03CC203F01CEC0BF008C000F009C076
:1055CE0001F00AC002F00BC003F0300E002641C2FB
:1055DE00E1FF42C2E2FF00C0E6FF0A0E046E000EBB
:1055EE00056E066E076E39C200F03AC201F03BC27C
:1055FE0002F03CC203F01CEC0BF000C039F201C00B
:10560E003AF202C03BF203C03CF2000E046E0318E5
:10561E0008E10450021805E10450011802E100509F
:10562E00000A01E105D0010E3F5F000E405BAFD7CF
:02563E00120058
:105640004E0E01014F6F000E506F270E0B6E0D0EA8
:105650000C6E260E0D6E0D2EFED70C2EFCD70B2ECB
:10566000FAD70000300E0201696F6A6B50EC0FF040
:10567000020E0B6E450E0C6EA90E0D6E0D2EFED792
:105680000C2EFCD70B2EFAD700000000300E0201C2
:10569000696F6A6B50EC0FF0820E0C6EDD0E0D6EB2
:1056A0000D2EFED70C2EFCD700000000300E02019C
:1056B000696F6A6B50EC0FF0820E0C6EDD0E0D6E92
:1056C0000D2EFED70C2EFCD700000000200E02018C
:1056D000696F6A6B50EC0FF0820E0C6EDD0E0D6E72
:1056E0000D2EFED70C2EFCD700000000280E020164
:1056F000696F010E6A6F50EC0FF0820E0C6EDD0EBA
:105700000D6E0D2EFED70C2EFCD700000000080EEB
:105710000201696F010E6A6F50EC0FF0820E0C6E81
:10572000DD0E0D6E0D2EFED70C2EFCD700000000F6
:10573000010E0201696F010E6A6F50EC0FF0030E4B
:105740000B6E8A0E0C6E550E0D6E0D2EFED70C2EA6
:10575000FCD70B2EFAD700000000060E0201696F7D
:10576000010E6A6F50EC0FF0820E0C6EDD0E0D6EA6
:105770000D2EFED70C2EFCD7000000000C0E0201EF
:10578000696F010E6A6F50EC0FF0820E0C6EDD0E29
:105790000D6E0D2EFED70C2EFCD70000000012005F
:1057A0000201396B3A6BC00E696F010E6A6F50ECE3
:1057B0000FF0290E0201696F6F0E6A6F000E6B6F9A
:1057C0002DEC10F0940E0201696F010E6A6F50EC1F
:1057D0000FF0B40E0201696F700E6A6F000E6B6FEE
:1057E0002DEC10F00D0E0B6EAF0E0C6EB60E0D6E96
:1057F0000D2EFED70C2EFCD70B2EFAD700000D0E67
:105800000B6EAF0E0C6EB60E0D6E0D2EFED70C2E5F
:10581000FCD70B2EFAD700000201396B3A6B7DECF6
:1058200021F0110E546F710E556F000E566FABECD8
:1058300021F00D0E0B6EAF0E0C6EB60E0D6E0D2E12
:10584000FED70C2EFCD70B2EFAD700000101C46B3B
:10585000C56B9D80D40E0201546F010E556F630E0F
:10586000566F000E576F020E586F000E596F4CECBA
:1058700021F0000E011802E1000E001806E1010EF1
:105880000201396F000E3A6F07D0000E0101C519F1
:1058900002E1000EC419DEE00101000EC51902E1AB
:1058A000010EC41905E139C200F03AC201F0D4D1A9
:1058B000E76BD40E0201696F010E6A6F50EC0FF0B6
:1058C000D40E0201696F010E6A6F67EC10F00D0EC5
:1058D0000B6EAF0E0C6EB60E0D6E0D2EFED70C2E8F
:1058E000FCD70B2EFAD70000940E696F010E6A6F79
:1058F00050EC0FF0A50E0201696F700E6A6F000E7A
:105900006B6F2DEC10F00D0E0B6EAF0E0C6EB60E15
:105910000D6E0D2EFED70C2EFCD70B2EFAD70000E5
:105920007DEC21F0EC0E546F700E556F000E566F2B
:10593000ABEC21F00D0E0B6EAF0E0C6EB60E0D6EB5
:105940000D2EFED70C2EFCD70B2EFAD7000001012E
:10595000C46BC56B9D80D40E0201546F010E556F50
:10596000660E566F000E576F080E586F000E596F77
:105970004CEC21F0000E011802E1000E001806E1C7
:10598000020E0201396F000E3A6F07D0000E0101BE
:10599000C51902E1000EC419DEE00101000EC519AF
:1059A00002E1010EC41905E139C200F03AC201F06A
:1059B00053D1E76BD40E0201696F010E6A6F50EC90
:1059C0000FF0D40E0201696F010E6A6F67EC10F0E0
:1059D0000D0E0B6EAF0E0C6EB60E0D6E0D2EFED7AD
:1059E0000C2EFCD70B2EFAD70000940E696F010E17
:1059F0006A6F50EC0FF0960E0201696F700E6A6FBD
:105A0000000E6B6F2DEC10F00D0E0B6EAF0E0C6ECA
:105A1000B60E0D6E0D2EFED70C2EFCD70B2EFAD720
:105A200000007DEC21F0310E546F700E556F000EAA
:105A3000566FABEC21F00D0E0B6EAF0E0C6EB60E6A
:105A40000D6E0D2EFED70C2EFCD70B2EFAD70000B4
:105A50000101E76BD40E0201696F010E6A6F50EC11
:105A60000FF0D40E0201696F010E6A6F67EC10F03F
:105A70000101C46BC56B9D80D40E0201546F010EF1
:105A8000556F590E566F000E576F090E586F000E66
:105A9000596F4CEC21F0000E011802E1000E0018C5
:105AA00006E1030E0201396F000E3A6F07D0000EB7
:105AB0000101C51902E1000EC419DEE00101000E6A
:105AC000C51902E1010EC41905E139C200F03AC25C
:105AD00001F0C2D0E76BD40E0201696F010E6A6F4C
:105AE00050EC0FF0D40E0201696F010E6A6F67EC83
:105AF00010F00D0E0B6EAF0E0C6EB60E0D6E0D2E61
:105B0000FED70C2EFCD70B2EFAD70000940E696F2F
:105B1000010E6A6F50EC0FF0C30E0201696F700E38
:105B20006A6F000E6B6F2DEC10F00D0E0B6EAF0E4A
:105B30000C6EB60E0D6E0D2EFED70C2EFCD70B2E56
:105B4000FAD700007DEC21F0E10E546F700E556F16
:105B5000000E566FABEC21F00D0E0B6EAF0E0C6EFF
:105B6000B60E0D6E0D2EFED70C2EFCD70B2EFAD7CF
:105B700000000101E76BD40E0201696F010E6A6F2C
:105B800050EC0FF0D40E0201696F010E6A6F67ECE2
:105B900010F00101C46BC56B9D80D40E0201546FDF
:105BA000010E556F500E566F000E576F080E586F4E
:105BB000000E596F4CEC21F0000E011802E1000EAE
:105BC000001803E10201394B3A2B0201040E396F30
:105BD000000E3A6F000E0101C51902E1010EC41951
:105BE00005E139C200F03AC201F036D00D0E0B6E5D
:105BF000AF0E0C6EB60E0D6E0D2EFED70C2EFCD712
:105C00000B2EFAD70000E76BD40E0201696F010E6C
:105C10006A6F50EC0FF0D40E0201696F010E6A6FCB
:105C200067EC10F009EC10F0050E0201396F000E60
:105C30003A6F0D0E0B6EAF0E0C6EB60E0D6E0D2E76
:105C4000FED70C2EFCD70B2EFAD700007DEC21F0EE
:0A5C500039C200F03AC201F0120060
:105C5A0039C204F03AC205F004C002F005C003F0EC
:105C6A00044A052A3BC200F03CC201F002013B4B48
:105C7A003C2B00C0E9FF01C0EAFF02C0E1FF03C0FC
:105C8A00E2FFEECFE6FF02C0E9FF03C0EAFFEE52F1
:0E5C9A0001E0E2D739C200F03AC201F0120078
:105CA800D40E0201696F010E6A6F50EC0FF0CEC17D
:105CB80054F2CFC155F239C256F23AC257F23BC23A
:105CC80058F2EEEC21F0CEC169F2CFC16AF267EC6E
:045CD80010F01200B6
:105CDC008AEC38F029EC25F089988292400EAF6E50
:105CEC00AC842EEC26F00C0E0201916F92EC0CF0B1
:105CFC000D0E0B6EAF0E0C6EB60E0D6E0D2EFED77E
:105D0C000C2EFCD70B2EFAD70000C80E0201546FD4
:105D1C006C0E556F000E566FABEC21F0B60E0201F7
:105D2C00546F6E0E556F000E566FABEC21F0000EDB
:105D3C000201546F6E0E556F000E566FABEC21F0D6
:105D4C001A0E0B6E5E0E0C6E6E0E0D6E0D2EFED7B9
:105D5C000C2EFCD70B2EFAD700008282EB0E010121
:105D6C00CE6F000ECF6F1F0E0201546F700E556F69
:105D7C00000E566FABEC21F089880201396BE3EC15
:105D8C0025F0200E396FE3EC25F0400E396FE3EC73
:105D9C0025F01A0E0B6E5E0E0C6E6E0E0D6E0D2E29
:105DAC00FED70C2EFCD70B2EFAD700000C0EC86EAB
:105DBC0063EC26F0500E396FE3EC25F089984E0E0B
:105DCC0001014F6F000E506F35DC010E0201696F3F
:105DDC00010E6A6F50EC0FF0800E0201696F010E1C
:105DEC006A6F50EC0FF0A30E0C6E550E0D6E0D2E4F
:105DFC00FED70C2EFCD7920E0201396F6F0E3A6F44
:105E0C00000E3B6F45EC25F0C00E696F010E6A6FFA
:105E1C0050EC0FF0600E0201396FE3EC25F07DECD5
:105E2C0021F00101D46BEB0ECE6F000ECF6F010E83
:105E3C000201696F010E6A6F50EC0FF0A30E0C6E2D
:105E4C00550E0D6E0D2EFED70C2EFCD7800E0201BA
:105E5C00696F010E6A6F50EC0FF0050E0201696F4D
:105E6C00710E6A6F000E6B6F2DEC10F0C00E0201FC
:105E7C00696F010E6A6F50EC0FF00B0E0201696F27
:105E8C00710E6A6F000E6B6F2DEC10F0940E020108
:105E9C00696F010E6A6F50EC0FF081B242D0680E40
:105EAC000201546F6F0E556F000E566FABEC21F064
:105EBC000201546B500E556FD3EC24F0010E02010D
:105ECC00546F590E556FD3EC24F0170E0201696F05
:105EDC0029EC0FF000C055F2020E546FD3EC24F0F5
:105EEC00030E0201546F020E556FD3EC24F0040E16
:105EFC000201546F140E556FD3EC24F0050E020101
:105F0C00546F050E556FD3EC24F00E0E0201696F21
:105F1C0029EC0FF000C055F2060E546FD3EC24F0B0
:105F2C0009D0860E0201546F700E556F000E566F1D
:105F3C00ABEC21F009EC10F01A0E0B6E5E0E0C6E31
:105F4C006E0E0D6E0D2EFED70C2EFCD70B2EFAD727
:105F5C0000007FEC26F0010E0201546F000E556F0D
:105F6C0038EC22F0700E0201396FE3EC25F06EEC88
:105F7C0026F0AB88AB889E6AA16AA46A9D6AA06A67
:105F8C00A36A9F6A9D8A9F8AD08EF19EF18CA26A29
:105F9C00F28CF28E080E4B6F000E4C6F9D80CD80F4
:105FAC00D0EC2BF000C04DF101C04EF1CD909D9086
:105FBC000D0E0B6EAF0E0C6EB60E0D6E0D2EFED7BB
:105FCC000C2EFCD70B2EFAD70000940E0201696F31
:105FDC00010E6A6F50EC0FF0A30E0C6E550E0D6E89
:105FEC000D2EFED70C2EFCD7800E006E800E0101FC
:105FFC004E19005C02E14D51040812E2CEC154F27C
:10600C00CFC155F2CF0E0201566F6E0E576F000EB8
:10601C00586F4DC159F24EC15AF2C9EC21F011D052
:10602C000201CEC154F2CFC155F2E60E566F6E0E80
:10603C00576F000E586F4DC159F24EC15AF2C9EC50
:10604C0021F0CEC169F2CFC16AF267EC10F00D0EEF
:10605C000B6EAF0E0C6EB60E0D6E0D2EFED70C2EFB
:10606C00FCD70B2EFAD7000001015D6B5E6B5F6BEA
:10607C00606BA46BA56BA66BA76BA86BA96BAA6BCB
:10608C00AB6B8988D26BD36B4D6B4E6BA26BA36BD6
:10609C0081B602D0D26BD36B81B01AD0000E4E19E0
:1060AC0002E1000E4D1914E1030E0B6E8A0E0C6EFC
:1060BC00550E0D6E0D2EFED70C2EFCD70B2EFAD7CF
:1060CC0000000000D24BD32B010E4D6F000E4E6F13
:1060DC0081A018D0000E4E1902E1010E4D1912E1EB
:1060EC00030E0B6E8A0E0C6E550E0D6E0D2EFED71A
:1060FC000C2EFCD70B2EFAD700000000D24BD32B62
:10610C004D6B4E6B000E0201321902E1010E31197A
:10611C001EE1D40E696F010E6A6FB3EC0FF009EC3F
:10612C0010F00101D451550A10E1E751230A0DE199
:10613C00200EE76FE86B3E0E0201396F6F0E3A6F5F
:10614C00000E3B6FABDD47EC27F07DEC21F0800EB1
:10615C000101D319006E800E005C02E1050ED25DC8
:10616C0097E30B0E0201396F700E3A6F000E3B6F06
:10617C0095DD0101A86BA96BAA6BAB6BAC6BAD6B1E
:10618C00AE6BAF6B5D6B5E6B5F6B606BBC6BBD6B5B
:10619C00BE6BBF6BC06BC16BC26BC36B640E4B6FC2
:1061AC00000E4C6FB86BB96BBA6BBB6BC46BC56B29
:1061BC00010EA26F000EA36F599DD26BD36B9F8003
:1061CC009F809D80CD80CD809D80F288010E020144
:1061DC00546F000E556F38EC22F025EC2AF055C1A7
:1061EC00B0F156C1B1F157C1B2F158C1B3F155C1BB
:1061FC00B4F156C1B5F157C1B6F158C1B7F10201AE
:10620C00010E546F000E556F38EC22F0800E006EAC
:10621C00800E0101D319005C02E1D2510508D8B0FF
:10622C0081D0D26BD36B5DC1BCF15EC1BDF15FC1DE
:10623C00BEF160C1BFF1C051BC5FC151BD5BC25169
:10624C00BE5BC351BF5BD40E0201696F010E6A6F56
:10625C0050EC0FF0410E0C6EEE0E0D6E0D2EFED7A7
:10626C000C2EFCD70000BCC100F0BDC101F0BEC1BA
:10627C0002F0BFC103F012EC0FF0660E046E660E56
:10628C00056E460E066E800E076E5EEC0AF000C0C0
:10629C009EF101C09FF102C0A0F103C0A1F1897869
:1062AC00CEC154F2CFC155F2A70E0201566F6F0E3C
:1062BC00576F000E586F00C059F201C05AF202C05D
:1062CC005BF203C05CF2C9EC21F0CEC169F2CFC124
:1062DC006AF267EC10F05DC1C0F15EC1C1F15FC143
:1062EC00C2F160C1C3F1BCC100F0BDC101F0BEC1BF
:1062FC0002F0BFC103F012EC0FF0290E046E5C0E1D
:10630C00056E670E066E810E076E5EEC0AF000C01D
:10631C00B8F101C0B9F102C0BAF103C0BBF101017F
:10632C005997E5D0BCC100F0BDC101F0BEC102F06F
:10633C00BFC103F012EC0FF0290E046E5C0E056E5B
:10634C00670E066E810E076E5EEC0AF000C0B8F1A7
:10635C0001C0B9F102C0BAF103C0BBF155C187F15C
:10636C0056C188F157C189F158C18AF10101B05168
:10637C00875FB151885BB251895BB3518A5B5DC158
:10638C0000F05EC101F05FC102F060C103F012ECDD
:10639C000FF0660E046E660E056E460E066E800ECF
:1063AC00076E5EEC0AF000C0A8F101C0A9F102C0B2
:1063BC00AAF103C0ABF1C00E0201696F010E6A6F46
:1063CC0050EC0FF0210E0C6E760E0D6E0D2EFED7CE
:1063DC000C2EFCD70000CEC154F2CFC155F2FD0EED
:1063EC000201566F6E0E576F000E586FA8C159F20E
:1063FC00A9C15AF2AAC15BF2ABC15CF2A4C15DF2B5
:10640C00A5C15EF2A6C15FF2A7C160F2C9EC21F092
:10641C00CEC169F2CFC16AF267EC10F00101598765
:10642C008A51000808E18951000805E188510008EB
:10643C0002E1875100085BE2D40E0201696F010E84
:10644C006A6F50EC0FF0410E0C6EEE0E0D6E0D2EB1
:10645C00FED70C2EFCD70000CEC154F2CFC155F2A2
:10646C00130E0201566F6F0E576F000E586F5DC101
:10647C0000F05EC101F05FC102F060C103F012ECEC
:10648C000FF000C035F201C036F202C037F203C083
:10649C0038F287C100F088C101F089C102F08AC1CD
:1064AC0003F012EC0FF000C004F001C005F002C0C4
:1064BC0006F003C007F035C200F036C201F037C257
:1064CC0002F038C203F05EEC0AF000C059F201C0D1
:1064DC005AF202C05BF203C05CF2C9EC21F0CEC1EF
:1064EC0069F2CFC16AF267EC10F00101598D000E10
:1064FC00C51902E1000EC41901E1F9D7C46BC56BD3
:10650C009D8059ADBCD0EB0ECE6F000ECF6F940EAC
:10651C000201696F010E6A6F50EC0FF0A30E0C6E46
:10652C00550E0D6E0D2EFED70C2EFCD7CEC154F28F
:10653C00CFC155F2BB0E0201566F6F0E576F000E96
:10654C00586FB8C159F2B9C15AF2BAC15BF2BBC1AA
:10655C005CF2C9EC21F0CEC169F2CFC16AF267ECF2
:10656C0010F03B0E01018B6FEB0ECE6F000ECF6F58
:10657C005DC139F25EC13AF25FC13BF260C13CF2DF
:10658C00CEC13DF2CFC13EF2AFEC2AF0CEC169F2E2
:10659C00CFC16AF2B3EC0FF08BC191F292EC0CF01C
:1065AC00A8C139F2A9C13AF2AAC13BF2ABC13CF283
:1065BC00670E02013D6F010E3E6F010E3F6F2AEC1C
:1065CC0028F0670E696F010E6A6FB3EC0FF08BC188
:1065DC0091F292EC0CF0A4C139F2A5C13AF2A6C129
:1065EC003BF2A7C13CF2670E02013D6F010E3E6FFC
:1065FC00020E3F6F2AEC28F0670E696F010E6A6F6E
:10660C00B3EC0FF08BC191F292EC0CF0B8C139F2F3
:10661C00B9C13AF2BAC13BF2BBC13CF2670E0201FE
:10662C003D6F010E3E6F020E3F6F2AEC28F08BC1BE
:10663C0091F292EC0CF0670E0201696F010E6A6F19
:10664C00B3EC0FF08BC191F292EC0CF09EC139F2CD
:10665C009FC13AF2A0C13BF2A1C13CF2670E02010C
:10666C003D6F010E3E6F010E3F6F2AEC28F0670E56
:10667C00696F010E6A6FB3EC0FF009EC10F00101B9
:10668C00D24BD32B000EA31902E1010EA21903E188
:10669C0081A601D0B4D5F298F29E030E0201546F7C
:1066AC00000E556F38EC22F0CF0E0201396F6F0ED1
:1066BC003A6F000E3B6F54EC2EF055C161F156C190
:1066CC0062F157C163F158C164F155C187F156C1EC
:1066DC0088F157C189F158C18AF10101B051875F26
:1066EC00B151885BB251895BB3518A5BA4C100F094
:1066FC00A5C101F0A6C102F0A7C103F0000E046E03
:10670C00000E056E610E066E8A0E076ED2EC04F05A
:10671C0000C035F201C036F202C037F203C038F2C5
:10672C0087C100F088C101F089C102F08AC103F071
:10673C0012EC0FF000C004F001C005F002C006F02E
:10674C0003C007F035C200F036C201F037C202F0C8
:10675C0038C203F05EEC0AF000C0B8F101C0B9F128
:10676C0002C0BAF103C0BBF100C039F201C03AF269
:10677C0002C03BF203C03CF2CEC13DF2CFC13EF2AF
:10678C00020E02013F6F2AEC28F0C00E696F010E59
:10679C006A6F50EC0FF0A30E0C6E550E0D6E0D2E95
:1067AC00FED70C2EFCD7CEC154F2CFC155F2650EDC
:1067BC000201566F700E576F000E586FA8C159F238
:1067CC00A9C15AF2AAC15BF2ABC15CF2C9EC21F0CF
:1067DC00CEC169F2CFC16AF267EC10F0940E696F0A
:1067EC00010E6A6F50EC0FF0A30E0C6E550E0D6E71
:1067FC000D2EFED70C2EFCD7CEC154F2CFC155F2C4
:10680C007D0E0201566F6F0E576F000E586FB8C198
:10681C0059F2B9C15AF2BAC15BF2BBC15CF2C9EC14
:10682C0021F0CEC169F2CFC16AF267EC10F0CEC193
:10683C0054F2CFC155F2760E566F700E576F000E94
:10684C00586FB0C159F2B1C15AF2B2C15BF2B3C1C7
:10685C005CF2C9EC21F0CEC169F2CFC16AF2B3ECA3
:10686C000FF0CEC154F2CFC155F2D20E566F700E4E
:10687C00576F000E586F61C159F262C15AF263C171
:10688C005BF264C15CF2C9EC21F0CEC169F2CFC1FC
:10689C006AF2B3EC0FF0CEC154F2CFC155F2760EC2
:1068AC00566F6E0E576F000E586F87C159F288C124
:1068BC005AF289C15BF28AC15CF2B8C15DF2B9C10E
:1068CC005EF2BAC15FF2BBC160F2C9EC21F0CEC17D
:1068DC0069F2CFC16AF2B3EC0FF009EC10F0CEC143
:1068EC0054F2CFC155F2FF0E0201566F6C0E576F6A
:1068FC00000E586FA8C159F2A9C15AF2AAC15BF295
:10690C00ABC15CF2A4C15DF2A5C15EF2A6C15FF29F
:10691C00A7C160F2B8C161F2B9C162F2BAC163F247
:10692C00BBC164F2C9EC21F0100E046E0E0E056EA4
:10693C00000E066E076E87C100F088C101F089C198
:10694C0002F08AC103F01CEC0BF000C024F201C071
:10695C0025F2280E0101CE250201356F000E010132
:10696C00CF210201366F0A0E046E000E056E97ECF5
:10697C0006F0300E002635C2E1FF36C2E2FF00C041
:10698C00E6FF290E0101CE250201356F000E010133
:10699C00CF210201366F0A0E046E000E056E24C262
:1069AC0000F025C201F097EC06F008C000F009C019
:1069BC0001F0300E002635C2E1FF36C2E2FF00C006
:1069CC00E6FF24C200F025C201F0100E046E0E0E7C
:1069DC00056ECAEC09F000500101875D006E015094
:1069EC008859016E00C0D2F101C0D3F13C0E046E87
:1069FC00000E056E97EC06F000C0D2F101C0D3F189
:106A0C002B0E0101CE250201356F000E0101CF21A5
:106A1C000201366F0A0E046E000E056E97EC06F03E
:106A2C00300E002635C2E1FF36C2E2FF00C0E6FFA1
:106A3C002C0E0101CE250201356F000E0101CF2174
:106A4C000201366F0A0E046E000E056ED2C100F004
:106A5C00D3C101F097EC06F008C000F009C001F0BA
:106A6C00300E002635C2E1FF36C2E2FF00C0E6FF61
:106A7C0024C200F025C201F0100E046E0E0E056E3D
:106A8C00CAEC09F000500101875D0201356F01501D
:106A9C00010188590201366FD2C100F0D3C101F057
:106AAC003C0E046E000E056ECAEC09F00050355D0C
:106ABC00006E01503659016E00C04DF101C04EF10F
:106ACC002E0E0101CE250201356F000E0101CF21E2
:106ADC000201366F0A0E046E000E056E97EC06F07E
:106AEC00300E002635C2E1FF36C2E2FF00C0E6FFE1
:106AFC002F0E0101CE250201356F000E0101CF21B1
:106B0C000201366F0A0E046E000E056E4DC100F0C8
:106B1C004EC101F097EC06F008C000F009C001F07E
:106B2C00300E002635C2E1FF36C2E2FF00C0E6FFA0
:106B3C00B70E0201396F000E3A6FCEC13BF2CFC1D6
:106B4C003CF22DEC2EF053C139F254C13AF2BCECAC
:106B5C0026F00101534B542B1EEC27F07DEC21F059
:106B6C00F28E000E321902E1010E311954E109ECDA
:106B7C0010F00101D451520A37E1D551450A34E1E4
:106B8C00D6514C0A31E1000ED11902E1030ED01995
:106B9C002BE1F70E0201546F6F0E556F000E566FFE
:106BAC00ABEC21F009EC10F002012F6B306B010102
:106BBC0054510201305D04E10101535102012F5D7A
:106BCC0013E22FC24DF130C24EF12FC239F230C256
:106BDC003AF272EC25F0AB0E696F000E6A6FB3ECF3
:106BEC000FF02F4B302BE3D70101D451550A11E193
:106BFC00E751230A0EE1200EE76FE86B530E0201FA
:106C0C00396F6F0E3A6F000E3B6F54EC2EF047EC61
:0A6C1C0027F07DEC21F0A5D7FFD78B
:1071140010EE26F0620E006E010E016E260EF66E63
:0E7124006C0EF76E000EF86E26EC26F01200D0
:106C260044696D616E004C756E6469004D617264F5
:106C360069004D65726372004A6575646900566540
:0A6C46006E64720053616D65640016
:096C50004F4B6C696E766F720007
:0A6C59004F4B7365746E616D6500AA
:036C63004F4B0094
:096C66004F4B73657450494E0058
:096C6F0030302F30302F3030009E
:096C780030303A30303A3030007F
:076C8100286E756C6C290000
:106C8800204E756D506167652032344C433235367D
:106C9800207265637570E972E965206465204C2788
:106CA800454550524F4D2064752050494320656E2C
:106CB800203078464520657420307846463D2000CF
:106CC8004D696B726F632070726F20362E343020DE
:106CD8003138463235382B2032344C433235362061
:106CE8002B204954205541525431202B2042542006
:076CF800484330360A0D008D
:106CFF00545464503D2520362E31663B4B6D733D09
:106D0F002520332E32663B566D6F793D2520332E6D
:106D1F0032663B44757265653D30304830304D30DA
:066D2F0030530D0A0000C4
:106D35000000007FCDCC4C7B0AD723786F120375FA
:106D450017B75171ACC5276EBD37066B95BF566732
:106D550077CC2B645F700961FFE65B5D08E53C3C21
:046D65006042221B4B
:106D69000000007F000020820000488500007A882A
:106D790000401C8C0050438F002474928096189612
:106D890020BC3E99286B6E9CF90215A0EC782DC1A8
:046D9900CAF249E20F
:106D9D000D0A204461746554696D653D202025738D
:106DAD002020206E657874204964782050616765D5
:106DBD005F456570726F6D203D2025203564202064
:036DCD000D0A00AC
:106DD0000100000008000000400000000002000068
:106DE00000100000008000000000040000002000EF
:106DF000000000010000000800000040000000004A
:106E000056657273696F6E203A20313430383230F3
:106E1000202063616C63756C206B6D7320656E2040
:0B6E2000666C6F7474616E740A0D00E4
:106E2B00010000000A00000064000000E8030000FD
:106E3B0010270000A086010040420F0080969800AA
:086E4B0000E1F50500CA9A3BC5
:106E53000A0D4D6973652061206C2768657572653D
:106E6300203A202573202020253264206361727329
:036E73000A0D0005
:106E760045636172743D25386C7520736563202007
:106E8600566974657373652025352E32660D0A00C2
:106E960001000000100000000001000000100000CA
:106EA60000000100000010000000000100000010BA
:106EB6002056656C6F20313846323538204D494BA7
:096EC600524F4320362E343000F7
:106ECF00496E6974204254204F4B2053746174658E
:076EDF003D25303264200064
:106EE600496E6974204254204241442053746174AF
:076EF600653D253032640008
:106EFD004E625464703D2520362E31662025332E8A
:066F0D003266204B6D000E
:106F130050756C73657320202F207365633D2520A6
:066F2300342E316620004F
:106F2900494E49542E4254204843303620424C455C
:056F390055202020009E
:106F3E0052654D6973652061206C274865757265D1
:056F4E00205254430035
:106F530052654D6973652061206C274865757265BC
:056F6300205254430020
:106F6800696E6974205254432070617220646566AA
:056F78006175742000AA
:106F7D0056697465737365206D6F792E3D202533C9
:056F8D002E3266200019
:106F92003138463235382032304D487A204D696BCF
:056FA200726F432000A6
:106FA7004E62546470202F204D6E203D2520352ED3
:046FB700316620001F
:106FBB0056697465737365204E6F773D20252035B8
:046FCB002E326600FC
:106FCF0053544F5020436F6D70746575722020209D
:046FDF00202020004E
:106FE300202020202020202020202020202020209E
:046FF300202020003A
:106FF70052656C6563747572652032344C43323563
:0470070036203A00F5
:10700B00436F6D70746575722052554E4E494E47E5
:04701B002020200011
:10701F0050726573656E746174696F6E203A200DDE
:02702F000A0055
:1070310041542B4E414D45484330362D3744363966
:0270410042000B
:10704300303132333435363738394142434445469B
:01705300003C
:1070540030313233343536373839616263646566CA
:01706400002B
:107065004E6220546450203D2025362E3166202066
:01707500001A
:1070760053746172743D25386C752073656309001D
:1070860052652D4C65637475726520525443200019
:0F70960045746170653A203320737572203400A1
:0F70A50045746170653A20322073757220340093
:0F70B40045746170653A20312073757220340085
:0F70C30045746170653A20342073757220340073
:0F70D20053746F703D25386C752073656309002A
:0B70E10041542B56455253494F4E00BE
:0B70EC0041542B50494E313233340028
:0770F700444154453A20001A
:0770FE0054494D453A200002
:0671050054494D453A001B
:06710B00444154453A0026
:03711100415400E6
:020000040030CA
:0D000100220F0EFFFF81FF0FC00FE00F4028
:0200000400F00A
:1000000056656C6F203138463235380D0A000000D5
:10001000436170746575722073757220524230208E
:10002000706F7572204170706172742E0D0A00003D
:10003000203436342070756C732F4B6D200D0A0000
:10004000203139394B6D73204D617869200D0A00DC
:10005000496E697420493243203430304B0D0A0018
:10006000496E69742044533133303720200D0A0023
:10007000496E69742042542D48433036200D0A00E1
:1000800072657365727665200D0AFFFFFFFFFFFF43
:100090002072657365727665204F4B20200D0A0033
:1000A0002072657365727665204F4B20200D0A0023
:1000B0002072657365727665204F4B20200D0A0013
:1000C0002072657365727665204F4B20200D0A0003
:1000D0002072657365727665204F4B20200D0A00F3
:1000E0002072657365727665204F4B20200D0A00E3
:1000F000646F6E27742075736520746869730000DF
:00000001FF
